:020000040800F2
:10000000E05C0020E101000819500008693A00088E
:10001000C1460008010A00086161000800000000F4
:10002000000000000000000000000000490100087E
:10003000FD0A0008000000008D0100082959000891
:10004000FB010008FB010008FB010008FB010008A0
:10005000FB010008FB010008FB010008FB01000890
:10006000FB010008FB010008FB010008FB01000880
:10007000FB010008A10A0008B10A0008C10A000833
:10008000FB010008FB010008D9070008FB0100087C
:10009000FB010008FB010008FB010008FB01000850
:1000A000FB010008FB010008FB010008FB01000840
:1000B000DD590008F9590008FB010008FB010008A0
:1000C000FB010008FB010008FB010008FB01000820
:1000D000FB010008BD600008FB0100085161000839
:1000E000FB010008FB010008FB010008FB01000800
:1000F000FB010008FB010008FB010008FB010008F0
:10010000FB010008FB010008FB010008FB010008DF
:10011000FB010008FB010008FB010008FB010008CF
:10012000FB010008FB010008FB010008FB010008BF
:10013000DFF810D000F004FB00480047A96B00086E
:10014000AFF30080E05C0020224B19680868B0E83B
:10015000F00F80F30988BFF36F8F4FF0000080F33A
:1001600011884EF00D0E7047000000000648006830
:10017000006880F3088862B661B6BFF34F8FBFF3A3
:100180006F8F00DF00BF00BF08ED00E0EFF30980D4
:10019000BFF36F8F0F4B1A6820E9F00F106008B59E
:1001A0004FF0500080F31188BFF34F8FBFF36F8F74
:1001B00007F07CFD4FF0000080F31188BDE8084097
:1001C00019680868B0E8F00F80F30988BFF36F8FF3
:1001D000704700BFD0050020EFF305807047000096
:1001E0000648804706480047FEE7FEE7FEE7FEE7D1
:1001F000FEE7FEE7FEE7FEE7FEE7FEE7DB59000865
:1002000031010008202A04DB203A21FA02F0002103
:10021000704721FA02F3D040C2F120029140084316
:100220001946704740EA01039B0703D009E008C95B
:10023000121F08C0042AFAD203E011F8013B00F8AB
:10024000013B521EF9D27047D2B201E000F8012BF7
:10025000491EFBD270470022F6E710B513460A4646
:1002600004461946FFF7F0FF204610BD421C10F867
:10027000011B0029FBD1801A7047F0B480EA01020B
:10028000D40F4200B2EB410F02D20246084611469B
:100290004A0042D0C30DDDB2C1F3C752AD1A202DC2
:1002A00035DAC1F3160141F4000204B15242C5F13E
:1002B000200602FA06F12A411044B3EBD05F23D0A6
:1002C000C4B1012DA0EBC35009DCF0BC4FF00042DB
:1002D00002EAC352DBB200F5000000F0A6B940000C
:1002E00000F1807000EBC350A0F1807040EAD17043
:1002F000490009E0490841EAC071A0EBC35000F58C
:100300000000400800EBC350F0BC00F085B961422A
:10031000012202EB4101001BF6E7F0BC704781F0BF
:100320000041AAE780F00040A7E780EA010210B58B
:1003300002F00043400022D04A001FD0010E01EB22
:100340001261C0F35600C2F3560240F4000042F4BA
:100350000002A0FB022000047F39140400D0401CDE
:1003600050EA124001D44000491EC2B20C0604EB10
:10037000D010401C4008802A02D003E0002010BDAD
:1003800020F00100002900DA0020184310BD30B42D
:1003900080EA010202F0004530F0004221F0004006
:1003A00013D090B1C30DD40DC2F31601C0F31600E3
:1003B000E41A41F4000140F400027D34914201D37B
:1003C000641C00E04900002C02DA30BC00207047B9
:1003D0004FF400000023914201D3891A03434008DF
:1003E0004FEA4101F7D151B1914202D14FF00041A2
:1003F00005E002D24FF0010101E06FF0010103EBD3
:10040000C450284430BC00F007B92DE9FE4F81EA02
:10041000030404F0004421F0004100944FF0000B6D
:1004200023F0004350EA01045ED052EA03045BD09B
:10043000C3F30A54C1F30A552C44A4F2F3340194D3
:10044000A0FB0254C1F3130141F48011C3F3130361
:1004500043F4801301FB024400FB034E840A970A15
:1004600044EA815447EA8357A4FB076802958D0A42
:1004700005FB07854FEA932C04FB0C542705029DCE
:100480004FEA065847EA1637B5EB08056EEB070C3E
:10049000870E920E47EA811742EA8312A7FB0201F8
:1004A000B6EB0B0164EB00042B0D43EA0C335E1832
:1004B00044EB1C50DA465146E7FB0201C5F3130436
:1004C0004FEA0B3343EA14534FEA0432019C43EAE8
:1004D0000603A4F10C040294009CCDE900B400F0E2
:1004E000E1F803B0BDE8F08F00200146F9E7C10F45
:1004F00080EAE0700844CA079623002100F095B80E
:1005000096230022114600F090B820F00040C10D63
:10051000C0F3160040F400007F2901DA0020704784
:10052000962903DCC1F19601C8407047963988408E
:100530007047C1F30A5210B5C1F3130140F2FF3303
:1005400041F480119A4201DA002010BD40F2334399
:100550009A42A2F2334203DC5242FFF753FE10BD2F
:10056000904010BD00F0004230F000400AD0C10DB4
:1005700001F56071C0F3160042EA0151C20840075C
:100580001143704700200146704701F0004330B42A
:1005900021F0004150EA010206D00A0DA2F5607276
:1005A000C1F31301002A02DC30BC00207047440F65
:1005B00044EAC104C100E01830BC00EBC25000F0B6
:1005C0002BB80000002801DBC0F10040002901DB4E
:1005D000C1F1004181427047002801DBC0F10040B9
:1005E000002901DBC1F100418842704730B50B465C
:1005F000014600202022012409E021FA02F59D4253
:1006000005D303FA02F5491B04FA02F52844151E26
:10061000A2F10102F1DC30BD0029A8BF7047401CE7
:10062000490008BF20F00100704710B4B0FA80FC08
:1006300000FA0CF050EA010404BF10BC704749B145
:10064000CCF1200421FA04F411FA0CF118BF0121B5
:1006500021430843A3EB0C01CB1D4FEA00614FEA95
:10066000102042BF002010BC704700EBC350104464
:100670000029A4BF10BC7047401C490008BF20F0EF
:10068000010010BC704710B5141E73F1000408DAA5
:10069000401C41F1000192185B411A4301D120F046
:1006A000010010BD2DE9F04D92469B4611B1B1FA03
:1006B00081F202E0B0FA80F22032904600F052F867
:1006C00004460F4640EA0A0041EA0B0153465A46E7
:1006D000084313D0114653EA010019D0C8F1400273
:1006E0005046FFF78FFD05460E4650465946424696
:1006F00000F038F8084305D0012004E020463946D0
:10070000BDE8F08D0020054346EAE0762C433743F0
:100710000A986305E40AA0EB08000022FD0A44EAF7
:1007200047540A3002D500200146E9E701051019B7
:100730006941DDE9084500196941BDE8F04DA2E7CE
:10074000064C074D06E0E06840F0010394E807001E
:1007500098471034AC42F6D3FFF7EEFCB88200089D
:10076000D8820008202A04DB203A00FA02F1002097
:1007700070479140C2F1200320FA03F319439040DF
:10078000704770B58C1810F8015B15F0070301D1A4
:1007900010F8013B2A1106D110F8012B03E010F8E4
:1007A000016B01F8016B5B1EF9D12B0705D4002307
:1007B000521E0DD401F8013BFAE710F8013BCB1AA9
:1007C000921C03E013F8015B01F8015B521EF9D59E
:1007D000A142D8D3002070BD10B5024800F05FFCE4
:1007E00010BD0000840F002070B50446002520686D
:1007F000806800F0010018B32068806820F00100D4
:100800002168886001F040FD054613E001F03CFDE1
:10081000401B02280ED92068806800F0010048B112
:10082000A06A40F01000A062E06A40F00100E062BF
:10083000012070BD2068806800F001000028E5D12B
:100840000020F6E738B50446002500200090206817
:10085000806800F0010078BB2068806840F00100EB
:1008600021688860194800681949B0FBF1F00090D0
:1008700002E00098401E009000980028F9D101F095
:1008800003FD054619E001F0FFFC401B022814D9C6
:100890002068806800F0010078B9A06A40F010007C
:1008A000A062E06A40F00100E06200BF002084F82E
:1008B000240000BF012038BD05E02068806800F0FA
:1008C00001000028DFD00020F5E70000CC05002063
:1008D00040420F0010B5184806F06AFD174908801D
:1008E000174806F065FD17490880144800884FF640
:1008F000FF71884202D01148008801E01248008848
:10090000114908800F4800884FF6FF71884202D0D5
:100910000C48008801E00D4800880C4908800A480E
:100920000088C0F30E000849088008480088C0F31A
:100930000E000649088010BD00180708D4000020EA
:1009400000200708D6000020E6000020E800002074
:10095000F0B597B006460D4601A803F0B5F800249F
:1009600012E004F50070854202D94FF4007700E0F0
:100970002F1B31193A461148FFF754FC3A460F49EC
:1009800001A803F0A1FC3C44AC42EAD301A90C4805
:1009900003F06CF8002407E00948005D0949615C38
:1009A000884200D002E0641C102CF5D300BF102C4C
:1009B00002D3012017B0F0BD0020FBE7002000208B
:1009C0001E28002000500708F0B50446187822F8C9
:1009D00010400025002004E032F810603544461C29
:1009E000F0B20A28F8DB0A20B5FBF0F0088018788E
:1009F000401C0A2690FBF6F706FB17001870F0BDA6
:100A000000BFFEE72DE9FC4707460D463846FFF7D5
:100A100077FD81462946FFF788FC04464FF08B415D
:100A2000FFF7B5FC064631462846FFF778FC8146BD
:100A300049463046FFF7ABFC04461549FFF775FC05
:100A40008046002419E0134A601C52F820104046EA
:100A5000FFF7C2FD10D80F4850F824104046FFF7AA
:100A6000B1FD09D20A2023460A4A0B49CDE90040CC
:100A7000404605F0F3FE04E0641C40F24720844247
:100A8000E1D300BF05480088FFF73AFDBDE8FC87C9
:100A90000000204134030020EC00002080050020ED
:100AA00010B5024800F0F2FE10BD000040490020E1
:100AB00010B5024800F0EAFE10BD0000FC4800201E
:100AC00010B5024800F0E2FE10BD0000B84800205A
:100AD00030B590F840500124AC40C56B6C600468A0
:100AE00063604468102C04D10468A2600468E1606B
:100AF00003E00468A1600468E26030BD704770B52F
:100B000003460024002010E00E5C451C4D5D46EAC3
:100B10000526851C4D5D46EA0546C51C4D5D46EA29
:100B2000056543F82450641C001D9042ECD370BD51
:100B300070B5034614460022002015E011F822503B
:100B40001D5431F82250C5F30726451C5E5551F857
:100B50002250C5F30746851C5E5551F822502D0ED4
:100B6000C61C9D55521C001DA042E7D370BD72B635
:100B700000BFFEE70021074AD1610749096941F03A
:100B80000401054A11611146096941F040011161F2
:100B900070470000D0490020002002400021074A91
:100BA000D1610749096941F00201054A1161114605
:100BB0004861096941F0400111617047D049002046
:100BC000002002400022054BDA61054A126942F01A
:100BD0000102034B1A61018070470000D0490020D8
:100BE0000020024000201E49C96801F0100139B1FF
:100BF0001C49C96941F002011A4AD16140F0100054
:100C00001749C96801F0040139B11649C96941F0B1
:100C10000101144AD16140F004001149C96901F091
:100C2000010169B10F49C96941F004010D4AD1615F
:100C300000BF0B49C96921F00101094AD16100BF18
:100C400000BF40F20111884206D10549C96921F06F
:100C50000101034AD16101E00149C86000BF70474A
:100C600000200240D049002070B5044601F00CFB82
:100C7000054609E0601C38B124B101F005FB401BBA
:100C8000A04201D9032070BD1248C06800F00100E5
:100C90000028EFD10F48C06800F0200020B100BF4D
:100CA00020200C49C86000BF0A48C06800F010004E
:100CB00048B90848C06900F0010020B90548C0687B
:100CC00000F0040018B1FFF78DFF0120DBE70020E2
:100CD000D9E7000000200240F0B503461C4600257D
:100CE0000026084607E010F8015B10F8016B45EAA2
:100CF000062724F8027B171EA2F1010C1FFA8CF2C2
:100D0000F1D1F0BD2DE9F04786B080460E46914600
:100D10004FF0000A00270025C6F30A0AA6EB0A07CF
:100D2000002005900190039701200490820239462B
:100D30001548FFF7D1FF00BF07E038F8150005EBB5
:100D40005A01114A22F811006D1C4D45F5D301F0EE
:100D5000CBF805A901A801F00DF800240BE00A4822
:100D600030F814C007EB440162460023012001F073
:100D700063F8601C84B2B4F5806FF0DB01F052F8C8
:100D800006B0BDE8F0870000001000202DE9F04714
:100D900081463A4800F0BEFB6421384800F0FAFA78
:100DA000364800F078F986B235493046FFF72AFE1A
:100DB0008046FFF7AAFB87B2324B334A33493846A5
:100DC000FFF702FE2D4800F0A5FB64212B4800F040
:100DD000E1FA2A4800F05FF985B22D480580B5B1E7
:100DE0002C48008800F4004010B12B48008802E035
:100DF000294800884042284485B240F68B60274944
:100E0000088008460088854201DB08460588244B97
:100E1000244A25492846FFF7D7FD184800F07AFBF9
:100E20006421164800F0B6FA144800F034F984B290
:100E30001E480480B4B11E48008800F4004010B180
:100E40001C48008802E01B4800884042204484B2CD
:100E500040F68B601849088008460088844201DB10
:100E600008460488154B164A16492046FFF7ACFD84
:100E7000024800F0E7FBBDE8F0870000840F002087
:100E800033335340DE000020B40F0020D800002090
:100E9000E2000020D4000020E60000207C050020B5
:100EA000DF000020C80F0020DA000020E40000204E
:100EB000D6000020E80000207E050020E000002091
:100EC000DC0F0020DC0000202DE9F041002500248B
:100ED0001EE0002600270CE0104A02EBC4029188B5
:100EE0000E4A52F8340004F0ABFB304486B2781C52
:100EF000C7B20A2FF0DB052E04DB0120A0402843F7
:100F0000C5B203E00020A0402843C5B2601CC4B2B3
:100F1000082CDEDB2846BDE8F0810000A081000837
:100F200002490968C1F3C300704700000C0C01407E
:100F30007047000038B5024600230020009000BF33
:100F400092F82400012801D1022038BD012082F846
:100F5000240000BF4868072812D21068406B0C7943
:100F6000641E04EB84051F24AC40A0430D796D1E64
:100F700005EB85050C68AC4020431468606327E0EE
:100F800048680D2812D21068006B0C79E41F04EB3E
:100F900084051F24AC40A0430D79ED1F05EB8505AA
:100FA0000C68AC4020431468206311E01068C06AEC
:100FB0000C790D3C04EB84051F24AC40A0430D7953
:100FC0000D3D05EB85050C68AC4020431468E062DC
:100FD00008680A2812D31068C0680C780A3C04EB31
:100FE00044050724AC40A0430D780A3D05EB4505B8
:100FF0008C68AC4020431468E0600FE01068006922
:101000000C7804EB44050724AC40A0430D7805EBB5
:1010100045058C68AC40204314682061086810289E
:1010200002D00868112827D1174C1068A0421ED1A1
:101030001068806800F40000F0B91068806840F41F
:1010400000001468A0600868102815D10F480068D7
:101050000F4CB0FBF4F000EB80004000009002E089
:101060000098401E009000980028F9D104E0906A92
:1010700040F020009062012300BF002082F824008D
:1010800000BF184661E7000000240140CC050020A5
:1010900040420F00704701460868C06C704770B549
:1010A0000446206805682068466806F0200020286D
:1010B0002DD105F00200022829D1A06A00F010000D
:1010C00018B9A06A40F40070A0622068806800F43B
:1010D0006020B0F5602F13D1207B88B9206840686C
:1010E00020F0200021684860A06A20F48070A0628F
:1010F000A06A00F4805018B9A06A40F00100A06214
:101100002046FFF7C7FF6FF012002168086006F065
:101110008000802839D105F00400042835D1A06A68
:1011200000F0100018B9A06A40F40050A0622068D6
:10113000806800F4E040B0F5E04F0DD020684068D2
:1011400000F48060D0B92068806800F46020B0F5B9
:10115000602F13D1207B88B92068406820F0800080
:1011600021684860A06A20F48050A062A06A00F460
:10117000807018B9A06A40F00100A0622046FFF715
:10118000D7FE6FF00C002168086006F04000402890
:101190000DD105F0010050B1A06A40F48030A0628A
:1011A000204600F0B5F86FF001002168086070BDBE
:1011B0002DE9F0410446002700250026A84614B971
:1011C0000120BDE8F081A06810B1207D00B100BF12
:1011D000A06A30B90020E06284F82400204600F0C4
:1011E00099F82046FFF700FB0746A06A00F01000C0
:1011F000002873D1002F7ED1A06A20F4885040F0DF
:101200000200A0623F4AD4E90001904208D1E0699F
:10121000B0F5402F02D14FF4002002E0E06900E079
:10122000E0690143207B41EA40000643A068B0F535
:10123000807F02D0A068012802D14FF4807000E0C6
:1012400000200543207D012811D1207B38B9A069F9
:10125000401E4FF4006141EA4030054307E0A06AB8
:1012600040F02000A062E06A40F00100E0622068E7
:10127000406820F4694028432168486020688068FD
:1012800021490840304321688860A068B0F5807F1C
:1012900002D0A068012802D14FF4807000E0002045
:1012A000B0F5807F03D1208A401E4FEA00582068A5
:1012B000C06A20F4700040EA08002168C862206813
:1012C000806812490840B04209D10020E062A06A5B
:1012D00020F0020040F00100A06211E00BE0A06AE3
:1012E00020F0020040F01000A062E06A40F001002F
:1012F000E062012704E0A06A40F01000A06201272C
:1013000038465EE7003C0140FDF7E1FFFE0E1FFF9F
:101310007047000010B586B004460020029003908C
:10132000049005901849206888422AD100BF1748C8
:10133000806940F40070154988610846806900F4AE
:101340000070019000BF00BF00BF0846806940F0F8
:10135000100088610846806900F01000019000BF0D
:1013600000BF072002900320039002A9084800F064
:10137000D3FD00220521122001F046F8122001F0D1
:1013800033F806B010BD00000024014000100240F8
:1013900000100140F8B504460D46002600200090DC
:1013A000002700F071FF06462068806800F4807016
:1013B00050B1A06A40F02000A06200BF002084F875
:1013C000240000BF0120F8BD2068406800F4807050
:1013D00020BB2068C06A00F47000F8B917E0681CF0
:1013E000A8B125B100F050FF801BA8420FD920689A
:1013F000006800F0020050B9A06A40F00400A0624A
:1014000000BF002084F8240000BF0320DBE7206831
:10141000006800F002000028E1D053E0022001F053
:1014200067F838490968B1FBF0F021680969364A64
:10143000114091B92168C9689211114069B92168B8
:101440000969324A114031B92168C96892111140C5
:1014500009B9142117E0292115E0216809692B4AEF
:10146000114021B92168C9689211114041B1216828
:101470000969274A114029B92168C968114009B989
:10148000542100E0FC2100FB01F718E0681C98B132
:1014900025B100F0F9FE801BA8420DD90098B84292
:1014A0000AD2A06A40F00400A06200BF002084F8C5
:1014B000240000BF032086E70098401C009000989D
:1014C000B842E3D36FF0120021680860A06A40F4CC
:1014D0000070A0622068806800F46020B0F5602F82
:1014E0000DD1207B58B9A06A20F48070A062A06A58
:1014F00000F4805018B9A06A40F00100A0620020FA
:1015000061E70000CC05002024499224922449126E
:101510004992240070B50446002500BF94F82400C9
:10152000012801D1022070BD012084F8240000BFF1
:101530002046FFF787F90546002D77D1A06A40F2D3
:101540000121884340F48070A0623C4920688842B1
:1015500008D13B48006800F4702008B9012002E07F
:10156000002000E0012078B1A06A20F48010A06281
:101570002068406800F4806000B3A06A20F4005046
:1015800040F48050A06219E0A06A40F48010A0628C
:101590002B49091F2068884203D0284920688842C7
:1015A00004D12748006800F4806000E0002028B1E2
:1015B000A06A20F4005040F48050A062A06A00F4B9
:1015C000805020B1E06A20F00600E06201E00020D7
:1015D000E06200BF002084F8240000BFC01E216824
:1015E00008602068806800F46020B0F5602F16D194
:1015F00012492068884208D11148006800F4702020
:1016000008B9012002E0002000E0012038B1206884
:10161000806840F4A000216888600CE006E0206843
:10162000806840F480102168886004E000BF0020DA
:1016300084F8240000BF284675E700000028014018
:101640000424014070B50446002500BF94F824002E
:10165000012801D1022070BD012084F8240000BFC0
:101660002046FFF7C1F805462DB9A06A20F488503E
:1016700040F00100A06200BF002084F8240000BFF9
:101680002846E8E70146002291F82100022808D008
:101690000420886300BF002081F8200000BF0120E3
:1016A00070470868006820F00E000B681860086832
:1016B000006820F001000B68186091F840300120AC
:1016C0009840CB6B5860012081F8210000BF0020BA
:1016D00081F8200000BF1046E2E7000070B5044624
:1016E000002594F82100022803D00420A0630125DE
:1016F000C1E02068006820F00E00216808602068C2
:10170000006820F00100216808605C492068884278
:1017100052D95A4978392068884201D1012047E0DE
:10172000564964392068884201D1102040E053496D
:1017300050392068884201D1801539E04F493C3941
:101740002068884201D1801432E04C492839206851
:10175000884202D14FF480302AE048491439206889
:10176000884202D14FF4801022E044492068884228
:1017700001D140041CE042492068884201D1012087
:1017800016E03F4914312068884201D110200FE053
:101790003B4928312068884201D1801508E038494A
:1017A0003C312068884201D1801401E04FF4803040
:1017B0003349091F086051E0304978392068884270
:1017C00001D1012047E02D4964392068884201D1C8
:1017D000102040E0294950392068884201D1801505
:1017E00039E026493C392068884201D1801432E032
:1017F000224928392068884202D14FF480302AE0FB
:101800001E4914392068884202D14FF4801022E02A
:101810001A492068884201D140041CE01849206818
:10182000884201D1012016E0154914312068884210
:1018300001D110200FE0124928312068884201D1DF
:10184000801508E00E493C312068884201D180149F
:1018500001E04FF48030094980394860012084F864
:10186000210000BF002084F8200000BF606B10B191
:101870002046616B8847284670BD0000800002400A
:10188000080402400146886B7047000070B50446AA
:10189000E06B05682068066894F8401004208840D2
:1018A0002840002875D006F004000028FAD02068EF
:1018B000006800F0200028B92068006820F00400CB
:1018C00021680860D5492068884254D9D3497839BD
:1018D0002068884201D1042049E0D0496439206859
:1018E000884201D1402042E0CC49503920688842EA
:1018F00001D100153BE0C9493C392068884202D13A
:101900004FF4804033E0C54928392068884202D12D
:101910004FF480202BE0C14914392068884202D15D
:101920004FF4800023E0BD492068884201D1C00403
:101930001DE0BB492068884201D1042017E0B84966
:1019400014312068884201D1402010E0B449283188
:101950002068884201D1001509E0B1493C31206876
:10196000884202D14FF4804001E04FF48020AC491E
:10197000091F086054E0A94978392068884201D1DC
:1019800004204AE0A54964392068884202D14020F9
:1019900043E04CE0A14950392068884201D100154C
:1019A0003BE09E493C392068884202D14FF4804098
:1019B00033E09A4928392068884202D14FF48020C8
:1019C0002BE0964914392068884202D14FF48000F8
:1019D00023E092492068884201D1C0041DE090496B
:1019E0002068884201D1042017E08D491431206815
:1019F000884201D1402010E089492831206888427E
:101A000001D1001509E086493C312068884202D1A5
:101A10004FF4804001E04FF48020804980394860D5
:101A2000E06A002802D02046E16A8847F4E094F892
:101A30004010022088402840002871D006F00200A3
:101A40000028FAD02068006800F0200040B9206823
:101A5000006820F00A0021680860012084F8210055
:101A60006E492068884254D96C4978392068884288
:101A700001D1022049E0694964392068884201D1D6
:101A8000202042E0654950392068884201D1401544
:101A90003BE062493C392068884202D14FF4005053
:101AA00033E05E4928392068884202D14FF4003083
:101AB0002BE05A4914392068884202D14FF40010B3
:101AC00023E056492068884201D180041DE0544932
:101AD0002068884201D1022017E051491431206862
:101AE000884201D1202010E04D49283120688842E9
:101AF00001D1401509E04A493C312068884202D1B1
:101B00004FF4005001E04FF400304549091F0860D0
:101B100054E0424978392068884202D102204AE0E4
:101B200057E03E4964392068884201D1202042E0D4
:101B30003A4950392068884201D140153BE0374985
:101B40003C392068884202D14FF4005033E03349D9
:101B500028392068884202D14FF400302BE02F4909
:101B600014392068884202D14FF4001023E02B4939
:101B70002068884201D180041DE0294920688842FC
:101B800001D1022017E0264914312068884201D192
:101B9000202010E0224928312068884201D14015D8
:101BA00009E01F493C312068884202D14FF40050BF
:101BB00001E04FF4003019498039486000BF00202F
:101BC00084F8200000BFA06A30B32046A16A88478D
:101BD00022E094F84010082088402840E0B106F048
:101BE0000800C8B12068006820F00E002168086075
:101BF00094F8401001208840E16B48600120A06308
:101C000084F8210000BF002084F8200000BF206B72
:101C100010B12046216B884770BD00008000024053
:101C2000080402400146002209B9012070471E4BFA
:101C3000086898420BD21D4B0868C01A1423B0FBE9
:101C4000F3F08000086419480838C8630AE0164BAE
:101C50000868C01A1423B0FBF3F08000086412482F
:101C60000838C863022081F821000868026843F63A
:101C7000F0708243D1E901031843CB6818430B6924
:101C800018434B6918438B691843CB6918430243C7
:101C90000868026000208863012081F8210000208C
:101CA00081F8200000BFC1E708040240080002409C
:101CB0002DE9F04104460D4616461F464FF0000838
:101CC00000BF94F82000012802D10220BDE8F08175
:101CD000012084F8200000BF94F8210001282CD1B5
:101CE000022084F821000020A0632068006820F012
:101CF0000100216808603B46324629462046FEF72F
:101D0000E7FEE06A30B12068006840F00E0021680C
:101D100008600BE02068006820F00400216808607B
:101D20002068006840F00A002168086020680068A8
:101D300040F001002168086006E000BF002084F840
:101D4000200000BF4FF002084046BFE770B50446D0
:101D500000F09AFA06462546681C10B1044800783F
:101D6000054400BF00F090FA801BA842FAD370BD72
:101D7000C80500202DE9F04104460E460127002544
:101D800000BF2648007E012802D10220BDE8F08174
:101D900001202249087600BF2068022813D14CF2A6
:101DA0005030FEF761FF90BB0120FEF7E3FE4CF2DE
:101DB0005030FEF759FF07461948006920F004002B
:101DC0001749086123E04CF25030FEF74DFFF0B99F
:101DD0004FF0FF303060A56812E02846FEF7DEFEC7
:101DE0004CF25030FEF740FF07460D48006920F0E6
:101DF00002000B4908610FB1356007E005F5006589
:101E0000D4E9021001EBC020A842E6D800BF00BF11
:101E100000200249087600BF3846B7E7D0490020C5
:101E2000002002400348006940F080000149086139
:101E300000207047002002402DE9FE4F05468B46EA
:101E400017469846012600240020029000BF24482F
:101E5000007E012802D10220BDE8FE8F012020492A
:101E6000087600BF4CF25030FEF7FEFE064686BBF9
:101E7000012D02D10120029006E0022D02D10220A4
:101E8000029001E00420029000241EE02201B946E5
:101E9000C24648465146FEF7B5F980B2019002208D
:101EA00000FB04B000900199FEF78CFE4CF250301C
:101EB000FEF7DAFE06460B48006920F001000949EA
:101EC000086106B104E0601CC4B202988442DDDB04
:101ED00000BF00BF00200249087600BF3046BBE7C4
:101EE000D04900200020024000200849096901F083
:101EF000800151B10649054A5160064951601146B9
:101F0000096901F0800101B1012070470020024001
:101F100023016745AB89EFCD2DE9F8470246002341
:101F20009C467BE14FF0010808FA03F4D1F80080E9
:101F300008EA0400A0427DD1DFF8F4A2D1F80480C1
:101F4000A8EB0A09D0453AD014DCB8F1030F50D001
:101F500009DCB8F1000F31D0B8F1010F1CD0B8F195
:101F6000020F49D120E0B8F1110F18D0B8F1120FCB
:101F700042D11EE0B9F5881F25D006DCB9F5803FB7
:101F800020D0B9F5801F37D11AE0B9F5001F18D05D
:101F9000B9F5041F30D117E0D1F80CC02DE0D1F80D
:101FA0000C8008F1040C28E0D1F80C8008F1080C32
:101FB00023E0D1F80C8008F10C0C1EE000BF00BF3C
:101FC00000BF00BF00BF00BFD1F80880B8F1000F0C
:101FD00002D14FF0040C0BE0D1F80880B8F1010FEA
:101FE00003D14FF0080C146102E04FF0080C54616B
:101FF00003E04FF0000C00E000BF00BFFF2801D855
:10200000904601E002F104084646FF2802D84FEA54
:10201000830803E0A3F108084FEA88084746D6F88A
:1020200000804FF00F0909FA07F928EA09080CFAAD
:1020300007F900E07AE048EA0908C6F80080D1F81C
:10204000048008F08058B8F1805F6FD100BFDFF8DE
:10205000E481D8F8188048F00108DFF8D891C9F871
:102060001880C846D8F8188008F00108CDF800801C
:1020700000BF00BF4FEAB9384FEA930958F829501A
:102080004FEA83784FEA18794FF00F0808FA09F8F9
:1020900025EA0805DFF8A081424502D14FF000088B
:1020A00024E0DFF89881424502D14FF001081DE09D
:1020B000DFF88C81424502D14FF0020816E0DFF8CC
:1020C0008481424502D14FF003080FE0DFF87881A8
:1020D000424502D14FF0040808E0DFF87081424524
:1020E00002D14FF0050801E04FF006084FEA83796E
:1020F0004FEA197908FA09F848EA0505DFF850812E
:102100004FEA930948F82950D1F8048008F4801860
:10211000B8F5801F0BD1DFF83C81D8F8008048EA81
:102120000008DFF83091C9F800800AE075E0DFF8B8
:102130002481D8F8008028EA0008DFF81891C9F84F
:102140000080D1F8048008F40018B8F5001F0ED103
:10215000DFF8008108F10408D8F8008048EA000898
:10216000DFF8F09009F10409C9F800800DE0DFF80C
:10217000E48008F10408D8F8008028EA0008DFF8B5
:10218000D49009F10409C9F80080D1F8048008F45A
:102190000038B8F5003F0ED1DFF8B880A8F1040888
:1021A000D8F8008048EA0008DFF8A890A9F10409EF
:1021B000C9F800800DE0DFF89C80A8F10408D8F889
:1021C000008028EA0008DFF88C90A9F10409C9F81A
:1021D0000080D1F8048008F48038B8F5803F0ED133
:1021E000DFF87080A8F10808D8F8008048EA0008F5
:1021F000DFF86090A9F10809C9F800800DE0DFF868
:102200005480A8F10808D8F8008028EA0008DFF810
:102210004490A9F10809C9F800805B1CD1F800803E
:1022200028FA03F8B8F1000F7FF47CAEBDE8F88718
:10223000000011100010024000080140000C014095
:10224000001001400014014000180140001C014032
:102250000800014008040140024693680B400BB19E
:10226000012000E00020704710B5C26821EA020397
:1022700002EA010443EA0443036110BD0AB10161AB
:1022800001E00B04036170470148006870470000DB
:10229000C005002003480068034909780844014943
:1022A00008607047C0050020C805002010B5084828
:1022B000006840F0100006490860032000F0E2F8D2
:1022C0000F2000F007F800F05FF8002010BD0000BC
:1022D000002002402DE9F04188B004460027B846AE
:1022E000002600BF2348C06940F002002149C861B0
:1022F0000846C06900F00200019000BF00BF02A9BB
:1023000003A800F0DFFA069F1FB900F003FB0546A3
:1023100002E000F0FFFA45001748B5FBF0F0A0F12D
:10232000010816481649086040F2E7311448C160B8
:10233000C0F80480002101618160816100F0C4FD6A
:10234000064696B90E4800F013FE06466EB91D20EB
:1023500000F04AF8102C07D2002221461D2000F080
:1023600053F80848046000E00126304608B0BDE894
:10237000F08100000010024040420F0000040040C5
:1023800084490020C405002008B500BF14488069B6
:1023900040F00100124988610846806900F00100A0
:1023A000009000BF00BF00BF0846C06940F08050E9
:1023B000C8610846C06900F08050009000BF00BFAF
:1023C00000220F21901E00F01FF800BF0549486849
:1023D00020F0E06040F00070486000BF08BD0000E1
:1023E000001002400000014001460846002809DBB9
:1023F00000F01F0301229A4043099B0003F1E023F0
:10240000C3F8002100BF70472DE9F05F80460D46FC
:102410001646002703F064FF074639462A4633462E
:1024200001F00700C0F1070ABAF1040F02D94FF01A
:10243000040A01E0C0F1070AD14600F1040ABAF12A
:10244000070F02D24FF0000A01E0A0F1030AD446C0
:102450004FF0010A0AFA09FAAAF1010A0AEA020A85
:102460000AFA0CFA4FF0010B0BFA0CFBABF1010B63
:102470000BEA030B4AEA0B042146404603F038FFFF
:10248000BDE8F09F00BF00F00702064B19684FF649
:10249000FF031940044B0B4343EA0221014B19602F
:1024A00000BF70470CED00E00000FA0500BF00BF60
:1024B00000BF00BF00BFBFF34F8F00BF00BF00BF12
:1024C0000948006800F4E06008490843001D064917
:1024D000086000BF00BF00BFBFF34F8F00BF00BF49
:1024E00000BF00BF00BFFDE70CED00E00000FA05F3
:1024F0002DE9F04706464FF000080025002700248C
:10250000A146042E37D004DC012E3CD0022E6CD123
:1025100060E0082E33D0102E67D13648446800683A
:1025200000F0807008B33448C4F38341475C04F47E
:10253000803078B12F484068C0F340402F4911F8EF
:10254000008004F4803040B12D48B0FBF8F000FB6F
:1025500007F502E02B4807FB00F52648406800F429
:102560008000B0F5800F01D1A94603E06800032187
:10257000B0FBF1F93AE000F0EDF9814636E000F009
:10258000E9F9814632E01B48046A04F44070B0F572
:10259000807F05D104F0020010B14FF4004918E02B
:1025A00004F44070B0F5007F07D11248406A00F093
:1025B000020010B149F640490BE004F44070B0F558
:1025C000407F06D10B48006800F4003008B14FF29C
:1025D00024490BE000F0AEF906494968C1F38131A6
:1025E000491C4900B0FBF1F900E000BF00BF4846BC
:1025F000BDE8F08700100240628200087282000885
:1026000000127A0000093D00F8B5044600260025B6
:10261000207800F0010000286BD000274348C069F3
:1026200000F0805070B900BF4048C06940F0805051
:102630003E49C8610846C06900F08050009000BF64
:1026400000BF01273A48006800F48070B0B93848EC
:10265000006840F4807036490860FFF715FE0646B2
:1026600006E0FFF711FE801B642801D90320F8BDA6
:102670002F48006800F480700028F2D02B48006AD0
:1026800000F440752DB3A08800F44070A84220D01B
:102690002648006A20F44075012026490860002081
:1026A00008602248056205F0010090B1FFF7ECFDDB
:1026B000064608E0FFF7E8FD801B41F288318842BA
:1026C00001D90320D3E71948006A00F0020000286E
:1026D000F0D01648006A20F440706168084313493E
:1026E0000862012F04D10846C06920F08050C861FB
:1026F00000BF207800F00200022807D10B48406894
:1027000020F44040A168084308494860207800F060
:102710001000102807D10548406820F48000616946
:102720000843024948600020A1E700000010024071
:10273000007000404004424270B504460D460CB99A
:10274000012070BD5A48006800F00700A8420ED270
:102750005748006820F0070028435549086008469C
:10276000006800F00700A84201D00120E9E72078C6
:1027700000F0020002281DD1207800F00400042897
:1027800005D14C48406840F4E0604A4948602078F0
:1027900000F00800082805D14648406840F4605021
:1027A000444948604348406820F0F000A16808436D
:1027B00040494860207800F0010078B36068012843
:1027C00006D13C48006800F4003090B90120B8E719
:1027D0006068022806D13748006800F0007040B9F0
:1027E0000120AEE73348006800F0020008B901207C
:1027F000A7E73048406820F00300616808432D498E
:102800004860FFF741FD064609E0FFF73DFD801BEC
:1028100041F28831884202D9032092E707E0254837
:10282000406800F00C006168B0EB810FEDD12048EA
:10283000006800F00700A8420ED91D48006820F08B
:10284000070028431A4908600846006800F007009E
:10285000A84201D0012074E7207800F00400042889
:1028600007D11448406820F4E060E168084311494A
:102870004860207800F00800082808D10D4840681A
:1028800020F46050216940EAC1000A49486000F024
:1028900061F808494968C1F30311074A515CC8400F
:1028A0000649086006480068FFF714FD002048E765
:1028B000002002400010024074820008CC05002075
:1028C000C40500200F2202600D4A526802F0030284
:1028D00042600B4A526802F0F0028260084A526875
:1028E00002F4E062C260064A526802F46052D20802
:1028F0000261044A126802F007020A607047000091
:1029000000100240002002400148006870470000AB
:10291000CC05002000B5FFF7F7FF04494968C1F373
:102920000221034A515CC84000BD00000010024073
:102930008482000800B5FFF7E7FF04494968C1F346
:10294000C221034A515CC84000BD00000010024093
:102950008482000870B5002100220024002300209A
:10296000134D696801F00C05F5B1042D02D0082D56
:1029700019D101E00F4819E00F4DC1F38346AB5D5B
:1029800001F4803555B10A4D6D68C5F340450B4ED5
:10299000725D084D5D43B5FBF2F402E0084D03FBA8
:1029A00005F4204602E000BF024800BF00BF70BD32
:1029B0000010024000127A00508200086082000875
:1029C00000093D00F8B504460CB90120F8BD207897
:1029D00000F00100002878D0F848406800F00C00B2
:1029E00004280CD0F548406800F00C00082811D1EC
:1029F000F248406800F48030B0F5803F0AD1EF48DB
:102A0000006800F4003000285FD0606800285CD1C6
:102A10000120DBE700BF6068B0F5803F06D1E748E2
:102A2000006840F48030E549086028E0606858B9E3
:102A3000E248006820F48030E049086008460068F9
:102A400020F4802008601AE06068B0F5A02F0BD158
:102A5000DA48006840F48020D849086008460068D9
:102A600040F4803008600AE0D448006820F48030E8
:102A7000D24908600846006820F48020086000BF42
:102A8000606888B1FFF700FC054606E0FFF7FCFB35
:102A9000401B642801D9032098E7C848006800F467
:102AA00000300028F2D010E0FFF7EEFB054606E00C
:102AB000FFF7EAFB401B642801D9032086E7BF48E3
:102AC000006800F400300028F2D1207800F0020005
:102AD000022857D1B948406800F00C0050B1B748FF
:102AE000406800F00C00082818D1B448406800F491
:102AF000803098B9B148006800F0020020B1206928
:102B0000012801D0012061E7AC48006820F0F800FE
:102B1000616940EAC100A949086033E02069E8B171
:102B20000120A7490860FFF7AFFB054606E0FFF765
:102B3000ABFB401B022801D9032047E79F480068F0
:102B400000F002000028F2D09C48006820F0F80055
:102B5000616940EAC1009949086013E00020984982
:102B60000860FFF791FB054606E0FFF78DFB401B71
:102B7000022801D9032029E79048006800F00200EC
:102B80000028F2D1207800F0080008282DD1A06993
:102B9000B8B101208B490860FFF776FB054606E0D7
:102BA000FFF772FB401B022801D903200EE7834880
:102BB000406A00F002000028F2D0012002F02CFD53
:102BC00013E000207F490860FFF75EFB054606E042
:102BD000FFF75AFB401B022801D90320F6E677488D
:102BE000406A00F002000028F2D1207800F00400D2
:102BF000042873D100277148C06900F0805070B973
:102C000000BF6E48C06940F080506C49C8610846FA
:102C1000C06900F08050009000BF00BF01276A48E3
:102C2000006800F48070B0B96748006840F48070B4
:102C300065490860FFF728FB054606E0FFF724FB1F
:102C4000401B642801D90320C0E65F48006800F4F7
:102C500080700028F2D000BFE068012806D15748F4
:102C6000006A40F001005549086227E0E06858B961
:102C70005248006A20F00100504908620846006A84
:102C800020F00400086219E0E06805280BD14B48E9
:102C9000006A40F00400494908620846006A40F0B2
:102CA000010008620AE04548006A20F0010043493B
:102CB00008620846006A20F00400086200BFE0686D
:102CC000A0B1FFF7E1FA054609E0FFF7DDFA401B86
:102CD00041F28831884202D9032077E622E0374862
:102CE000006A00F002000028EFD012E0FFF7CCFAF3
:102CF000054608E0FFF7C8FA401B41F288318842D8
:102D000001D9032062E62D48006A00F00200002885
:102D1000F0D1012F05D12948C06920F08050274902
:102D2000C86100BFE069C8B32448406800F00C00E7
:102D3000082860D0E069022848D1002020490866B0
:102D4000FFF7A2FA054606E0FFF79EFA401B0228AD
:102D500001D903203AE61948006800F00070002805
:102D6000F2D1206AB0F5803F07D11448406820F4C2
:102D70000030A168084311494860D4E908010843BC
:102D80000E49496821F4741108430C494860012038
:102D90000B490866FFF778FA054607E03DE0FFF7C4
:102DA00073FA401B022801D903200FE6034800688C
:102DB00000F000700028F2D02FE000000010024068
:102DC000000042428004424200700040002014494A
:102DD0000866FFF759FA054606E0FFF755FA401B6B
:102DE000022801D90320F1E50E48006800F00070C8
:102DF0000028F2D111E0E069012800D1E6E5094898
:102E0000466806F48031206A814204D106F47011CC
:102E1000606A814201D00120D8E50020D6E500009B
:102E200000004242001002407047704730B5024631
:102E30000B4600BF92F83C00012801D1022030BDB2
:102E4000012082F83C0000BF022082F83D0010689B
:102E500044681068816824F070041868044310689E
:102E60004460144D1068A84213D0134D1068A84256
:102E70000FD01068B0F1804F0BD0104D1068A842F1
:102E800007D00F4D1068A84203D00E4D1068A8421D
:102E900005D121F08001586801431068816001204C
:102EA00082F83D0000BF002082F83C0000BF00BF58
:102EB000C5E70000002C0140003401400004004040
:102EC00000080040000C004010B504460CB9012079
:102ED00010BD94F83D0028B9002084F83C0020463D
:102EE00000F026F8022084F83D00211D206802F041
:102EF0008BFD012084F8460000BF84F83E000121CC
:102F00003F200155402001554120015500BF00BF21
:102F1000012084F8420043200155442001554520FA
:102F2000015500BF012084F83D000020D0E70000DB
:102F300038B504462068B0F1804F15D100BF0B486A
:102F4000C06940F001000949C8610846C06900F045
:102F50000100009000BF00BF002205211C20FFF7E8
:102F600053FA1C20FFF740FA38BD00000010024061
:102F7000014691F83D00012801D001207047022050
:102F800081F83D000868C06840F001000B68D86017
:102F9000164B0868984213D0154B086898420FD01A
:102FA0000868B0F1804F0BD0124B0868984207D0E8
:102FB000114B0868984203D0104B086898420CD116
:102FC0000868806800F00702062A0CD008680068CC
:102FD00040F001000B68186005E00868006840F0E8
:102FE00001000B6818600020C8E70000002C0140B9
:102FF000003401400004004000080040000C004084
:103000002DE9F04104460D46002700BF94F83C002E
:10301000012802D10220BDE8F081012084F83C00A3
:1030200000BF022084F83D002068866826F07706FD
:1030300026F47F46206886602868502833D00CDC50
:10304000202850D004DC00284BD0102851D149E072
:10305000302849D040284CD139E060282DD0702844
:1030600007D0B0F5805F03D0B0F5005F41D10DE02F
:1030700041E0D5E902136A68206802F013FD206878
:10308000866846F077062068866034E0D5E902134A
:103090006A68206802F006FD2068806840F480407D
:1030A0002168886027E0EA686968206802F00EFD00
:1030B0005021206802F001FD1DE0EA68696820687F
:1030C00002F017FD6021206802F0F7FC13E0EA68C7
:1030D0006968206802F0FAFC4021206802F0EDFCEB
:1030E00009E000BF00BF00BF2968206802F0E5FCCE
:1030F00001E0012700BF00BF012084F83D0000BFB0
:10310000002084F83C0000BF384684E7704710B5C3
:10311000044620680069C0F34000D8B12068C06848
:10312000C0F34000B0B16FF00200216808610120D7
:1031300020772068806900F0030018B12046FFF76F
:10314000E5FF05E0204600F0ADF8204600F0ABF8C2
:103150000020207720680069C0F38000D8B1206883
:10316000C068C0F38000B0B16FF00400216808614E
:10317000022020772068806900F4407018B1204652
:10318000FFF7C4FF05E0204600F08CF8204600F071
:103190008AF80020207720680069C0F3C000D8B109
:1031A0002068C068C0F3C000B0B16FF008002168AB
:1031B0000861042020772068C06900F0030018B17E
:1031C0002046FFF7A3FF05E0204600F06BF82046FD
:1031D00000F069F80020207720680069C0F3001033
:1031E000D8B12068C068C0F30010B0B16FF0100013
:1031F00021680861082020772068C06900F44070C9
:1032000018B12046FFF782FF05E0204600F04AF89B
:10321000204600F048F8002020772068006900F080
:10322000010058B12068C06800F0010030B16FF0B3
:10323000010021680861204600F036F82068006926
:10324000C0F3C01058B12068C068C0F3C01030B1DE
:103250006FF08000216808612046FFF7E5FD2068D7
:103260000069C0F3801058B12068C068C0F38010B6
:1032700030B16FF0400021680861204600F020F86E
:1032800020680069C0F3401058B12068C068C0F3DE
:10329000401030B16FF02000216808612046FFF730
:1032A000C4FD10BD7047704710B50446034920683F
:1032B000884201D1FEF7EEFF10BD0000000400407F
:1032C0007047704710B5044600BF00BF21680C313D
:1032D00051E8001F21F4907021680C3141E8000290
:1032E000002AF3D100BF00BF00BF2168143151E8AC
:1032F000001F21F001002168143141E80002002A7A
:10330000F3D100BF206B01280ED100BF00BF2168A0
:103310000C3151E8001F21F0100021680C3141E808
:103320000002002AF3D100BF2068406900F040008D
:1033300000B300BF00BF2168143151E8001F21F025
:1033400040002168143141E80002002AF3D100BF97
:10335000E06B78B10020E16B4863E06BFEF792F917
:1033600040B1E06BFEF78EFA202803D11020606494
:10337000032010BD0020E085202084F842000020BA
:10338000206300BFF5E770B504460025206840695A
:10339000C0F3C01594F84100212817D1B5B100BF82
:1033A00000BF2168143151E8001F21F0800021681E
:1033B000143141E80002002AF3D100BFA06B10B124
:1033C000A06BFEF75FF9204602F08BFC2068406995
:1033D000C0F3801594F84200222817D1B5B100BF80
:1033E00000BF2168143151E8001F21F0400021681E
:1033F000143141E80002002AF3D100BFE06B10B1A4
:10340000E06BFEF73FF9204602F025FC002070BD7E
:10341000704700002DE9F84F0446206805682068D1
:10342000C668206847694FF00009CA4605F00F09D1
:10343000B9F1000F0AD105F0200038B106F02000E4
:1034400020B1204602F060FCBDE8F88FB9F1000F12
:103450007BD007F0010018B906F49070002874D0F2
:1034600005F0010030B106F4807018B1606C40F0D6
:103470000100606405F0040030B107F0010018B1EC
:10348000606C40F00200606405F0020030B107F0AB
:10349000010018B1606C40F00400606405F00800A1
:1034A00048B106F0200010B907F0010018B1606CB7
:1034B00040F008006064606C002845D005F02000F2
:1034C00028B106F0200010B1204602F01DFC206853
:1034D0004069C0F3801A606C00F0080010B9BAF1BE
:1034E000000F2CD0204602F0B6FB2068406900F0A7
:1034F000400000B300BF00BF2168143151E8001F35
:1035000021F040002168143141E80002002AF3D183
:1035100000BFE06B50B17748E16B4863E06BFEF7AA
:10352000DDF888B1E06B416B88470DE02046FFF77E
:103530006FFF09E009E02046FFF76AFF04E020463C
:10354000FFF766FF002060647EE7206B012877D1DB
:1035500005F01000002873D006F010000028FAD003
:1035600000BF00200090206800680090206840683C
:10357000009000BF00BF2068406900F040000028B4
:103580005FD0E06B006840681FFA80F8B8F1000F68
:1035900055D0A08D404552DDA4F82E80E06B8069A7
:1035A000202843D000BF00BF21680C3151E8001F24
:1035B00021F4807021680C3141E80002002AF3D127
:1035C00000BF00BF00BF2168143151E8001F21F087
:1035D00001002168143141E80002002AF3D100BF44
:1035E00000BF00BF2168143151E8001F21F04000E6
:1035F0002168143141E80002002AF3D100BF2020E5
:1036000084F842000020206300BF00BF21680C3115
:1036100051E8001F21F0100021680C3141E8000240
:10362000002AF3D100BFE06BFEF72CF802206063A4
:10363000A08DE28D801A81B22046FFF742FE03E79B
:1036400042E0A08DE18D401A1FFA80F8E08DD0B3E2
:10365000B8F1000F37D000BF00BF21680C3151E82E
:10366000001F21F4907021680C3141E80002002A0B
:10367000F3D100BF00BF00BF2168143151E8001F23
:1036800021F001002168143141E80002002AF3D141
:1036900000BF202084F842000020206300BF00BF4C
:1036A00021680C3151E8001F21F0100021680C3115
:1036B00041E80002002AF3D100BF022060634146C6
:1036C0002046FFF7FEFDBFE605F0800030B106F0B2
:1036D000800018B1204602F077FCB5E605F0400006
:1036E00030B106F0400018B1204602F0EAFAABE62D
:1036F00000BFA9E61B5B000810B504460CB9012009
:1037000010BDA06900B100E000BF94F8410028B9E5
:10371000002084F84000204600F02AF8242084F895
:1037200041002068C06820F400502168C86020462D
:1037300002F068FB2068006920F49040216808616D
:103740002068406920F02A00216848612068C0682C
:1037500040F400502168C86000206064202084F894
:10376000410084F842000020606300BFC8E7000009
:1037700010B586B004460020029003900490059096
:103780006249206888426AD100BF6148806940F47C
:1037900080405F4988610846806900F4804001905C
:1037A00000BF00BF00BF0846806940F00400886188
:1037B0000846806900F00400019000BF00BF481572
:1037C0000290022003900320059002A95148FEF7C1
:1037D000A3FB4FF48060029000200390049002A9A4
:1037E0004C48FEF799FB4C484C4908600020486063
:1037F00000214A4881608021C1600021016141614E
:103800008161C161FEF70EFA08B1FDF7B0F900BFA2
:103810004248E063446200BF3F48143840490860B2
:103820001020486000213E4881608021C160002155
:10383000016141618161C161FEF7F4F908B1FDF7F1
:1038400096F900BF3648A063446200BF00220521FC
:103850002520FEF7D9FD2520FEF7C6FD54E03149AD
:103860002068884250D100BF2948C06940F48020B8
:103870002749C8610846C06900F48020019000BF54
:1038800000BF00BF0846806940F008008861084614
:10389000806900F00800019000BF00BF0815029089
:1038A000022003900320059002A91F48FEF734FB75
:1038B0004FF40060029000200390049002A91A487F
:1038C000FEF72AFB14482838184908600020486091
:1038D0000021164881608021C160002101614161A1
:1038E0008161C161FEF79EF908B1FDF740F900BFA3
:1038F0000E48E063446200BF002205212720FEF746
:1039000083FD2720FEF770FD06B010BD0038014092
:10391000001002400008014058000240B848002052
:10392000FC48002000480040000C014040490020B5
:1039300070B504460D46164694F8420020280BD177
:1039400005B10EB9012070BD002020633246294622
:10395000204602F0D5FAF6E70220F4E76FF02001E6
:1039600002681160891002681160704770472DE984
:10397000F84F04460E46174699464FF0000A94F851
:10398000410020284AD106B117B90120BDE8F88FBF
:1039900000206064212084F84100FEF775FC824617
:1039A000A784E784A068B0F5805F04D1206910B9CE
:1039B0000025B04602E035464FF000081BE05346B4
:1039C000002280212046CDF8009002F02DFB08B1A6
:1039D0000320DBE745B9B8F80000C0F30800216810
:1039E000486008F1020803E02878216848606D1CEF
:1039F000E08C401EE084E08C0028E0D15346002299
:103A000040212046CDF8009002F00EFB08B10320C3
:103A1000BCE7202084F841000020B7E70220B5E78A
:103A200010B5034693F84100202813D101B10AB91B
:103A3000012010BD19629A84DA8400205864212084
:103A400083F841001868C06840F080001C68E0609E
:103A50000020EEE70220ECE76FF020010268116021
:103A6000891002681160704700BFFEE72DE9FC4134
:103A700006460C46082204F110016846FDF758F886
:103A8000208AC0F3C505382D02D2C5F1380001E007
:103A9000C5F1780007463A460A49204600F014FC72
:103AA00008226946204600F00FFC102221463046CD
:103AB000FDF73EF858220021204600F051FCBDE8F9
:103AC000FC81000070000020002242610261054973
:103AD0000160054941600349C94381600249C94306
:103AE000C16070470123456789ABCDEF2DE9F043F5
:103AF00091B080468946D8F80040D8F80450D8F8EC
:103B00000860D8F80C704022494601A8FCF7F7FF7E
:103B100005EA060027EA0501084301990844FE4921
:103B200008440444E00140EA54642C4404EA0500DB
:103B300026EA0401084302990844F8490844074466
:103B4000380340EA1757274407EA040025EA07012B
:103B5000084303990844F24908440644700440EAC3
:103B6000D6363E4406EA070024EA060108430499D3
:103B70000844EC4908440544A80540EA9525354425
:103B800005EA060027EA0501084305990844E649C5
:103B900008440444E00140EA54642C4404EA05006B
:103BA00026EA0401084306990844E049084407440A
:103BB000380340EA1757274407EA040025EA0701BB
:103BC000084307990844DA4908440644700440EA67
:103BD000D6363E4406EA070024EA0601084308995F
:103BE0000844D44908440544A80540EA95253544CD
:103BF00005EA060027EA0501084309990844CE4969
:103C000008440444E00140EA54642C4404EA0500FA
:103C100026EA040108430A990844C84908440744AD
:103C2000380340EA1757274407EA040025EA07014A
:103C300008430B990844A0F524404F38064470040B
:103C400040EAD6363E4406EA070024EA0601084365
:103C50000C990844BA4908440544A80540EA95254A
:103C6000354405EA060027EA050108430D99084492
:103C7000B44908440444E00140EA54642C4404EA92
:103C8000050026EA040108430E990844AE49084499
:103C90000744380340EA1757274407EA040025EA97
:103CA000070108430F990844A849084406447004D2
:103CB00040EAD6363E4406EA070024EA06010843F5
:103CC00010990844A24908440544A80540EA9525EE
:103CD000354405EA070026EA07010843029908442B
:103CE0009C4908440444600140EAD4642C4404EA3A
:103CF000060025EA06010843079908449649084446
:103D00000744780240EAD757274407EA050024EA27
:103D1000050108430C990844904908440644B0033F
:103D200040EA96463E4406EA040027EA04010843B6
:103D3000019908448A4908440544280540EA153594
:103D4000354405EA070026EA0701084306990844B6
:103D5000844908440444600140EAD4642C4404EAE1
:103D6000060025EA060108430B9908447E490844E9
:103D70000744780240EAD757274407EA050024EAB7
:103D80000501084310990844784908440644B003E3
:103D900040EA96463E4406EA040027EA0401084346
:103DA00005990844724908440544280540EA153538
:103DB000354405EA070026EA070108430A99084442
:103DC0006C4908440444600140EAD4642C4404EA89
:103DD000060025EA060108430F990844664908448D
:103DE0000744780240EAD757274407EA050024EA47
:103DF0000501084304990844604908440644B00397
:103E000040EA96463E4406EA040027EA04010843D5
:103E1000099908445A4908440544280540EA1535DB
:103E2000354405EA070026EA070108430E990844CD
:103E3000544908440444600140EAD4642C4404EA30
:103E4000060025EA06010843039908444E49084440
:103E50000744780240EAD757274407EA050024EAD6
:103E60000501084308990844484908440644B0033A
:103E700040EA96463E4406EA040027EA0401084365
:103E80000D990844424908440544280540EA15357F
:103E9000354485EA06007840069908443D490844BF
:103EA0000444200140EA14742C4484EA0500704064
:103EB00009990844384908440744F80240EA57572A
:103EC000274487EA040068400C99084433490844B1
:103ED0000644300440EA16463E4486EA0700604045
:103EE0000F9908442E4908440544E80540EA552541
:103EF000354485EA06007840029908442949084477
:103F00000444200140EA14742C4484EA0500704003
:103F100005990844244949E078A46AD756B7C7E808
:103F2000DB702024EECEBDC1AF0F7CF52AC68747DB
:103F3000134630A8019546FDD8988069AFF7448BA9
:103F4000BED75C892211906B937198FD8E4379A640
:103F50002108B44962251EF640B340C0515A5E267E
:103F6000AAC7B6E95D102FD65314440281E6A1D842
:103F7000C8FBD3E7E6CDE121D60737C3870DD5F4DB
:103F8000ED145A4505E9E3A9F8A3EFFCD9026F67E0
:103F90008A4C2A8D4239FAFF81F6718722619D6D24
:103FA0000C38E5FD44EABEA4A9CFDE4B0844074423
:103FB000F80240EA5757274487EA04006840089906
:103FC0000844A74908440644300440EA16463E44E3
:103FD00086EA070060400B990844A249084405445A
:103FE000E80540EA5525354485EA060078400E99F3
:103FF00008449D4908440444200140EA14742C44B8
:1040000084EA05007040019908449849084407442F
:10401000F80240EA5757274487EA040068400499A9
:104020000844934908440644300440EA16463E4496
:1040300086EA07006040079908448E490844054411
:10404000E80540EA5525354485EA060078400A9996
:104050000844894908440444200140EA14742C446B
:1040600084EA050070400D990844844908440744D7
:10407000F80240EA5757274487EA0400684010993D
:1040800008447F4908440644300440EA16463E444A
:1040900086EA07006040039908447A4908440544C9
:1040A000E80540EA5525354465EA07007040019966
:1040B0000844754908440444A00140EA94642C442F
:1040C00064EA0600684008990844704908440744B7
:1040D000B80240EA9757274467EA050060400F9905
:1040E00008446B4908440644F00340EA56463E44FF
:1040F00066EA040078400699084466490844054485
:10410000680540EAD525354465EA070070400D99F9
:104110000844614908440444A00140EA94642C44E2
:1041200064EA06006840049908445C49084407446E
:10413000B80240EA9757274467EA050060400B99A8
:104140000844574908440644F00340EA56463E44B2
:1041500066EA04007840029908445249084405443C
:10416000680540EAD525354465EA0700704009999D
:1041700008444D4908440444A00140EA94642C4496
:1041800064EA060068401099084448490844074416
:10419000B80240EA9757274467EA0500604007994C
:1041A0000844434908440644F00340EA56463E4466
:1041B00066EA040078400E9908443E4908440544E4
:1041C000680540EAD525354465EA07007040059941
:1041D0000844394908440444A00140EA94642C444A
:1041E00064EA060068400C990844344908440744CE
:1041F000B80240EA9757274467EA050060400399F0
:1042000008442F4908440644F00340EA56463E4419
:1042100066EA040078400A9908442A49084405449B
:10422000680540EAD5253544D8F800002044C8F890
:104230000000D8F804002844C8F80400D8F80800A2
:104240003044C8F80800D8F80C003844C8F80C000E
:104250004022002101A800F083F811B0BDE8F083EE
:10426000604BBBF670BCBFBEC67E9B28FA27A1EA96
:104270008530EFD4051D880439D0D4D9E599DBE623
:10428000F87CA21F6556ACC4442229F497FF2A4348
:10429000A72394AB39A093FCC3595B6592CC0C8FD8
:1042A0007DF4EFFFD15D84854F7EA86FE0E62CFEA4
:1042B000144301A3A111084E827E53F735F23ABD93
:1042C000BBD2D72A91D386EB2DE9F0470446884626
:1042D0001546208AC0F3C509206900EBC50020619E
:1042E000B0EBC50F02D26069401C6061606900EBF1
:1042F00055716161C9F14007BD421BD304F118013A
:1043000001EB09003A46414600F020F804F118019B
:104310002046FFF7EBFB3E4605E008EB0601204692
:10432000FFF7E4FB403606F13F00A842F5D34FF01B
:10433000000900E00026AA1B08EB060104F118039F
:1043400003EB090000F002F8BDE8F08710B5034662
:10435000002002E00C5C1C54401C9042FAD310BDBB
:1043600010B50346002001E01954401C9042FBD3D5
:1043700010BD00000EB500200090019002901E4874
:104380001E49086081151D488160002101730121CB
:10439000017581614FF46021C161002017494860B7
:1043A000032116480161FCF703FF08B1FCF7DFFBAE
:1043B0000A200090012001900720029069460F48D2
:1043C000FCF7B8FD08B1FCF7D2FB0B2000900220EF
:1043D000019069460948FCF7ADFD08B1FCF7C7FB41
:1043E0000C2000900320019069460448FCF7A2FDD0
:1043F00008B1FCF7BCFB0EBD00240140840F002077
:1044000008B500BF1248406940F0010010494861FA
:104410000846406900F00100009000BF00BF002284
:1044200005210D20FDF7F0FF0D20FDF7DDFF002237
:1044300005210E20FDF7E8FF0E20FDF7D5FF002235
:1044400005210F20FDF7E0FF0F20FDF7CDFF08BD90
:104450000010024000B59DB01C22184916A8FBF7B9
:10446000E1FE002116A802F062FC154908601C223A
:1044700012491C310FA8FBF7D5FE00210FA802F04E
:1044800056FC104908601C220C49383108A8FBF77B
:10449000C9FE002108A802F04AFC0B4908601C2252
:1044A0000649543101A8FBF7BDFE002101A802F026
:1044B0003EFC064908601DB000BD0000E081000818
:1044C000C4000020C8000020CC000020D000002044
:1044D00000B585B00020019002900390049000BFC9
:1044E0003A48806940F01000384988610846806980
:1044F00000F01000009000BF00BF00BF08468069B8
:1045000040F0200088610846806900F0200000909B
:1045100000BF00BF00BF0846806940F0040088610A
:104520000846806900F00400009000BF00BF00BF93
:104530000846806940F0080088610846806900F0FC
:104540000800009000BF00BF002241F2790120481E
:10455000FDF794FE4FF6F87001900320029001A938
:104560001C48FDF7D9FCFF20019000200290039029
:1045700001A91948FDF7D0FC41F279000190012012
:104580000290002003900220049001A91048FDF73A
:10459000C3FC4EF2863001900320029001A90C4822
:1045A000FDF7BAFC4FF4194001900320029001A9D5
:1045B0000948FDF7B1FC042001900320029001A9F5
:1045C0000648FDF7A9FC05B000BD00000010024040
:1045D000000C01400010014000080140001401409F
:1045E00000B587B0002003900490059006900190DC
:1045F00002904FF080401549086040F21F3048603B
:1046000000211248816041F63F71C16000210161C3
:1046100080218161FEF758FC08B1FCF7A8FA4FF43D
:104620008050039003A90948FEF7EAFC08B1FCF7A3
:104630009EFA00200190029001A90448FEF7F6FBC3
:1046400008B1FCF794FA07B000BD00003433002035
:1046500010B50B480B4908604FF416504860002114
:1046600008488160C16001610C21416100218161C4
:10467000C161FFF741F808B1FCF779FA10BD0000FD
:10468000003801402848002010B50B480B4908604D
:104690004FF416504860002108488160C1600161F4
:1046A0000C21416100218161C161FFF725F808B14A
:1046B000FCF75DFA10BD0000004800407048002083
:1046C00000BFFEE710B586B0FE480078012831D162
:1046D0000621FD4801F0DAFFFB498979FA4AD279CF
:1046E00041EA02218842F2D1F84800880A2821DAFA
:1046F000F5480078F649097888421CD1F24840789C
:10470000032818D1F0488078A8B9EF48C07801286C
:1047100011D1ED48007970B9EB48407901280AD1F0
:1047200007200090EB48037802220321E848008824
:1047300002F04EFF11E2E4480078E549097888422A
:104740001CD1E1484078032818D1DF488078A8B907
:10475000DD48C078022811D1DB48007970B9DA4809
:10476000407901280AD107200090DB480378022213
:104770000321D748008802F02BFFDBE7D2480078FE
:10478000D349097888421CD1CF484078032818D1F2
:10479000CD488078A8B9CC48C078032811D1CA4840
:1047A000007970B9C848407901280AD107200090E3
:1047B000CA48038802220321C548008802F008FF86
:1047C000B8E7C1480078C249097888421CD1BE4880
:1047D0004078032818D1BC488078A8B9BA48C07876
:1047E000042811D1B848007970B9B7484079012838
:1047F0000AD107200090BA48038802220321B44856
:10480000008802F0E5FEFCE3AF480078B049097883
:1048100088421CD1AC484078032818D1AA48807837
:10482000A8B9A948C078052811D1A748007970B95E
:10483000A548407901280AD107200090A94803889B
:1048400002220321A248008802F0C2FED9E39E485A
:1048500000789F49097888421FD19B4840780328F7
:104860001BD199488078C0B99748C078012814D1E5
:104870009548007988B99448407902280DD10920DB
:1048800095490978CDE90010924803780422032164
:104890008F48008802F006FFB3E38B4800788C490C
:1048A0000978884222D18848407803281ED186485A
:1048B0008078D8B98448C078012817D18248007917
:1048C000A0B981484079032810D10B218348008882
:1048D000814A1278CDE9002002917E4803780622B1
:1048E00003217B48008802F07BFD8AE3764800784C
:1048F00077490978884225D173484078032821D127
:1049000071488078F0B97048C07801281AD16E4893
:104910000079B8B96C484079042813D10D2170484A
:1049200002886E4800886C4B1B78CDE90030CDE9D9
:10493000022168480378082203216548008802F0B4
:1049400097FD5EE36048007861490978884228D184
:104950005D484078032824D15B48807808BB5A48DA
:10496000C07801281DD158480079D0B956484079FF
:10497000052816D10F215B48028859480088574BFB
:104980001B88CDE90130CDE9032153480078009020
:10499000504803780A2203214D48008802F0BCFDEC
:1049A0002FE3494800784A49097888421FD1464890
:1049B000407803281BD144488078C0B94248C07869
:1049C000022814D14048007988B93F48407902282C
:1049D0000DD1092041490988CDE900103E480378EE
:1049E000042203213A48008802F05CFE09E33648BD
:1049F000007837490978884222D133484078032823
:104A00001ED131488078D8B92F48C078022817D1F4
:104A10002D480079A0B92C484079032810D10B21EA
:104A20002F4800882D4A1288CDE9002002912A489B
:104A30000378062203212648008802F0D1FCE0E238
:104A40002148007822490978884225D11E484078BB
:104A5000032821D11C488078F0B91B48C07802286F
:104A60001AD119480079B8B917484079042813D1E8
:104A70000D211C4802881A480088184B1B88CDE974
:104A80000030CDE9022114480378082203211048A0
:104A9000008802F0EDFCB4E20B4800780C4909787C
:104AA000884232D10848407803282ED106488078C1
:104AB00058BB0548C078032827D10348007920BB9C
:104AC000014811E0850500207C3B00208605002080
:104AD000B6000020C0000020C1000020DA00002045
:104AE000DC000020D8000020407902280DD10920E8
:104AF000FE490988CDE90010FD48038804220321FE
:104B0000FC48008802F0CEFD7BE2FB480078F949C2
:104B10000978884222D1F848407803281ED1F64807
:104B20008078D8B9F448C078032817D1F2480079C2
:104B3000A0B9F1484079032810D10B20EF4909882A
:104B4000EA4A1288CDE900210290E948038806224A
:104B50000321E848008802F043FC52E2E64800786E
:104B6000E449097888421FD1E348407803281BD1E3
:104B7000E1488078C0B9E048C078042814D1DE4804
:104B8000007988B9DC48407902280DD10920DB4939
:104B90000988CDE90010D548038804220321D548AF
:104BA000008802F07FFD2CE2D3480078FA281BD160
:104BB000D1484078032817D1CF488078A0B9CE4893
:104BC000C078AA2810D1CC48007968B9CA48407981
:104BD000012809D107200090C6480388022203213A
:104BE000FA2002F0F5FC0CE2C3480078C1490978CC
:104BF000884224D1C0484078032820D1BE4880781C
:104C000050281CD1BC48C078C8B9BB480079B0B99D
:104C1000B9484079022812D10921B948008880B2E8
:104C2000CDE90001B64800684FF6FF7101EA104374
:104C300004220321AF48008802F034FDE1E1AE48D0
:104C40000078AC490978884237D1AB4840780328CE
:104C500033D1A948807850282FD1A748C07802289E
:104C60002BD1A548007940BBA3484079022824D124
:104C7000A44802F041FE0921A348008880B2CDE992
:104C80000001A14800684FF6FF7101EA10430422B9
:104C900003219848008802F005FD9B48008840EAFF
:104CA00000209A4908800846008880380880964885
:104CB0000068803896490860A3E18F4800788D49E4
:104CC0000978884220D18C48407803281CD18A4832
:104CD0008078502818D18848C078042814D1864894
:104CE000007988B98448407901280DD1854802F0BF
:104CF00023FE0720009087480388022203217D4875
:104D0000008802F065FC7CE17B48007879490978ED
:104D1000884244D178484078032840D1764880784A
:104D200050283CD17448C078052838D172480079A1
:104D3000A0BB71484079082831D16E480078764987
:104D400008700320487010208870002011E073491B
:104D500031F810100912032202EB40026E4B9954F5
:104D60006E4911F81020032101EB4001491C5A54EF
:104D7000401C0828EBDB1321674801F087FC044640
:104D80006549CC7420120875192315226448FEF772
:104D9000EEFD01F0B3FC02F0E5FA32E1FFE7564820
:104DA000007854490978884229D153484078062828
:104DB00025D15148807810BB4F48C07802281ED1B9
:104DC0004D480079D8B94C49487902F0E5FC0522F4
:104DD0004949544801F0C6F947484079464C24797E
:104DE00040EA04234448C078434CA47840EA0422B3
:104DF000414841783F48008802F020FC01E13E48EC
:104E000000783C490978884229D13B4840780628F7
:104E100025D13948807810BB3748C0780A281ED180
:104E200035480079D8B934484079012817D1002293
:104E300031493D4801F096F92F4840792E4C2479AC
:104E400040EA04232C48C0782B4CA47840EA042282
:104E5000294841782748008802F0F0FBD1E0264835
:104E6000007824490978884229D1234840780628C7
:104E700025D12148807810BB1F48C0780B281ED14F
:104E80001D480079D8B91C484079012817D1002263
:104E90001949264801F066F917484079164C2479DB
:104EA00040EA04231448C078134CA47840EA042252
:104EB000114841780F48008802F0C0FBA1E00E487D
:104EC00000780C49097888424DD10B484078062873
:104ED00049D10948807858BB0748C0780C2842D18E
:104EE0000548007920BB0449487922E0DC00002015
:104EF000DA000020B60000207C3B0020D800002013
:104F0000BC000020003007083C00002018000020F2
:104F100024000020400000202E3000209A060020AF
:104F20002848002000080708001807080020070884
:104F300019E002F067FC05223349344801F012F908
:104F400031484079304C247940EA04232E48C07817
:104F50002D4CA47840EA04222B4841782C48008844
:104F600002F06CFB4DE02848007829490978884216
:104F700025D125484078062821D123488078F0B9EA
:104F80002148C078AA281AD11F480079B8B905224B
:104F90001D49204801F0E6F81B4840791A4C247955
:104FA00040EA04231848C078174CA47840EA042249
:104FB000154841781648008802F040FB21E012486D
:104FC000007813490978884217D10F48407806289D
:104FD00013D10D48807880B90B48C078CC280CD10B
:104FE00009480079A52808D1074840795A2804D1F2
:104FF00001F084FBFDF75AFA03E001F07FFB02F0B9
:10500000B1F906B010BD00007C3B0020001007087D
:10501000B60000200000070800BFFEE7FEB5002034
:10502000FE490870FE48407AFD49097A40EA0120AD
:10503000FC490880FA48C078F949897840EA01209B
:10504000F9490880F9480588F94903C9CDE9010102
:10505000F348C079F74908704FF48061F648FBF7D0
:10506000FAF84FF48061F548FBF7F5F8F14800785D
:10507000012804D002287CD004287BD12CE22822ED
:10508000E7490A31EE48FBF7CDF88021E4480A30C1
:1050900001F06CFBEB490880E81EE149095C281F20
:1050A000DF4A105C41EA0020E74908800020E74918
:1050B0000860E4480088E449098888427DD10024DA
:1050C0000AE0E3482044017904F10A00D44A105C64
:1050D000814200D002E0641C582CF2DB00BF322C6D
:1050E0006CDA00240FE00A2000EB4400CC49085C95
:1050F0000B2101EB4401CA4A515C40EA0120CE4930
:1051000021F81400641C192CEDDB1922D049091D6B
:10511000C948FBF7F7FD322001F049FB0120CD49DA
:105120000860CB491B31CC4802F02CF9C948006813
:1051300068B3C948007800F00F0042F2107148438C
:10514000C549497801F00F0101EB4102C2EBC111E1
:1051500000EBC100C049897801F00F0101EBC102E9
:1051600002EB011100EB8100BB49C97801F00F018E
:1051700001E0BEE029E201EB810100EB4100B6490C
:10518000097901F00F010844B449086022E0B248EF
:10519000007800F00F004FF47A714843AE49497827
:1051A00001F00F0101EBC10202EB011100EB8100E4
:1051B000A949897801F00F0101E080E061E001EB8D
:1051C000810100EB4101A448C07800F00F000844C1
:1051D000A2490860A1480068A1490860A14801F0FF
:1051E000EFFAFCF781FE9E4800239E4902680120E9
:1051F000FCF722FEFCF716FE96480068F8B1102274
:10520000934921319848FBF767FD08229749964852
:10521000FBF778FD00200FE0934931F810104FF4B0
:105220007F4202EA0121904A32F8102041EA12211D
:105230008D4A22F81010401C0828EDDB1EE01022D9
:10524000834920318848FBF747FD08228749864873
:10525000FBF758FD00200FE0834931F810104FF4A0
:105260007F4202EA0121804A32F8102041EA1221ED
:105270007D4A22F81010401C0828EDDB7C48734959
:1052800008604FF480616648FAF7E5FF502001F0AE
:105290008EFA78488079009076484079754E367954
:1052A00040EA06237348C078724EB67840EA062278
:1052B000704841787048008802F034FA0EE04FF4EC
:1052C00080615748FAF7C7FF01A8FAF7CFFF86B207
:1052D0006423324601A96948FEF749FB4FF4806117
:1052E0005548FAF7B8FF4FF480615448FAF7B3FF16
:1052F0006CE1634802F000FB614802F01DFB802175
:1053000047480A3001F032FA4E490880E81E444905
:10531000095C281F424A105C01EB00204A490880C2
:105320005848008881B2404800888030814203D1CB
:1053300001205549087002E0002053490870514887
:10534000008880B238490988884213D04E480078D6
:1053500080B1354800888038334908804948006862
:105360006FF30F0009880843464908600846006843
:1053700036490860334800883349098888424BD150
:10538000012211464148FCF779FF0120FCF7DEFCC1
:10539000002201213D48FCF771FF00240FE00A20A4
:1053A00000EB44001E49085C0B2101EB44011C4A40
:1053B000515C40EA0120204921F81400641C402C73
:1053C000EDDB4022214801681B48FBF79BFC1F488E
:1053D000006880301D490860084600682C49086054
:1053E000084600684FF6FF7101EA1040294908801D
:1053F0002748008848800B4800888880032220497D
:105400002448FBF77FFC4FF480610548FAF723FF3F
:10541000012211461D483FE05DE0000084050020A8
:105420007C33002016000020180000208605002094
:105430009881000804000020BA060020BA0A002063
:10544000380600201E00002020000020240000203C
:105450007AF0070834000020800600202800002091
:1054600058000020004807089A060020005007084E
:10547000000004087C3B0020B600002028480020E3
:10548000003007083C00002054000020000C0140C0
:105490003800002048000020FCF7F0FE0120FCF757
:1054A00055FC002201214A48FCF7E8FE4948807972
:1054B000009048484079474E367940EA06234548EF
:1054C000C078444EB67840EA0622424841784248C5
:1054D000008802F027F979E08021404801F046F980
:1054E0003F490880E81E3D490A39095C281F3B4AAC
:1054F0000A3A105C01EB00203A49088038480088DD
:105500000988884250D1082237493848FBF7E4FB24
:1055100000200FE0354931F810104FF47F4202EAC5
:105520000121324A32F8102041EA12212F4A22F892
:105530001010401C0428EDDB2D492C4801F0F8F830
:105540002C4801F03DF9FCF7CFFC294800232949FC
:1055500002680220FCF770FCFCF764FC2648016836
:105560002648FBF7F5F9264908600846006810B19F
:1055700000F08CF828E023A118480A3800F09CFEBF
:105580000646502001F013F9B2B214490A392148F5
:10559000FEF746FA02E00120FCF7D8FB1D4890F820
:1055A00041002128F7D00FE0502001F000F901A8B8
:1055B000FAF75CFE86B26423324601A91548FEF76D
:1055C000D6F9502001F0F3F800E000BF00BFFEBDA7
:1055D000000C01407C3B0020B600002086330020F8
:1055E0001E0000202000002088F007080600002090
:1055F000BC000020004007085800002000000408FC
:1056000030000020636865636B3D6572726F720DD8
:105610000A0000002848002008B508490968C908A0
:105620004FF47A72B1FBF2F14143009100BF00BF29
:1056300000994A1E00920029F9D108BDCC0500202E
:1056400070B504460D4629462046FCF705FE08B90C
:10565000012070BD0020FCE708B509480949086031
:105660000846008880B2ADF8020008460068000CC9
:10567000ADF80000022204496846FBF743FB08BD71
:10568000BBBB55552C0000207AF0070808B54FF039
:10569000AA30194908600846008880B2ADF80000B9
:1056A0000846008880B2ADF8020008460068009005
:1056B000042212496846FBF725FB00BF00BF00BF6C
:1056C00000BF00BFBFF34F8F00BF00BF00BF0C483B
:1056D000006800F4E0600B490843001D08490860B9
:1056E00000BF00BF00BFBFF34F8F00BF00BF00BFB0
:1056F00000BF00BFFDE700002C0000207AF0070883
:105700000CED00E00000FA0500BF012001F0FEFAF8
:10571000012211460B48FCF7B1FD0120FCF716FBF6
:10572000002201210748FCF7A9FDFBF7CDFB064944
:105730000870FBF7F5FB054908700548FBF726FBE9
:10574000E3E70000000C0140C0000020C100002081
:10575000840F002000BF012001F0D8FAFBE700BF52
:10576000012001F0D3FAFBE738B50222424968462E
:10577000FBF7B2FABDF80200BDF8001040EA0140A4
:105780003E4908603E4800683E4908604FF4806129
:105790003D48FAF760FD3D4802F04AF83748006896
:1057A000B0F1AA3F08D0B0F1BB3F04D0384908445B
:1057B000002850D142E05BE0314800683149086080
:1057C000084601683348FBF7C3F80546F5B12D4894
:1057D00030490268304801F059F95020FCF7B6FA18
:1057E0002EA1294800F068FD0446A2B2264930489F
:1057F000FEF716F902E00120FCF7A8FA2C4890F811
:1058000041002128F7D0FFF727FF16E029A11E4805
:1058100000F052FD0446502000F0C9FFA2B21A4920
:105820002348FEF7FDF802E00120FCF78FFA20483C
:1058300090F841002128F7D038BD00BF1148016819
:105840001548FBF785F828B1002000F074FD1248D8
:1058500001F0A0F90CE00B4801680F48FBF778F85D
:1058600028B1002000F067FD0B4801F093F9E3E751
:1058700000BF00BFE0E700007AF0070860000020EA
:1058800028000020580000207C3300200048070832
:105890004544AAAA00000408000002085570677277
:1058A00061646520636F6D706C65746564000000F1
:1058B00028480020636865636B6661696C000000BE
:1058C00000BF012001F022FA1248007801281ED101
:1058D000114800888E281AD110480078104909789C
:1058E000884214D10D484078102810D18C210D48E1
:1058F00000F0CCFE094991F88C10084A92F88D20EE
:1059000041EA0221884202D1FFF788FBD9E7FEF77E
:10591000D9FED6E784050020860500207C3B0020C8
:10592000B60000207C33002010B500BF502080F36B
:105930001188BFF34F8FBFF36F8F00BF02F006FBDC
:1059400018B14FF080500449086000BF002080F378
:10595000118800BF10BD000004ED00E000B595B057
:1059600028210BA8FAF777FC142106A8FAF773FC94
:1059700018216846FAF76FFC01200B9000040C9088
:1059800000200D9001200F9002201290C10313916E
:10599000002114910BA8FDF715F808B1FBF7E7F803
:1059A0000F2006900220079080200890C0000990E8
:1059B00000200A90002106A8FCF7BEFE08B1FBF704
:1059C000D6F802200090400302906846FCF71CFEC7
:1059D00008B1FBF7CCF815B000BD704710B54FF417
:1059E00080510348FCF740FC0248FDF790FB10BDD6
:1059F000000C01403433002010B50248FDF787FB4E
:105A000010BD00008449002010B50268204B984268
:105A10000ED0204B98420BD0B0F1804F08D01E4BD7
:105A2000984205D01D4B984202D01D4B984203D19D
:105A300022F070024B681A43154B98420ED0154B5A
:105A400098420BD0B0F1804F08D0134B984205D04C
:105A5000124B984202D0124B984203D122F440726A
:105A6000CB681A4322F080034C6943EA04020260C7
:105A70008B68C3620B688362054B984202D0054B6A
:105A8000984201D10B6903630123436110BD0000FB
:105A9000002C014000340140000400400008004098
:105AA000000C004030B50C46816821F47F4142EA89
:105AB000032525432943816030BD0A46816821F0D2
:105AC000700142F0070319438160704730B50B46FF
:105AD0001446026A056A25F001050562816921F014
:105AE000F00141EA041122F00A021A4381610262C4
:105AF00030BD30B50B461446026A056A25F0100524
:105B00000562816921F4704141EA043122F0A0026A
:105B100042EA03128161026230BD70B505466C6ACB
:105B20000020E085E0842046FDF772FC70BD70B572
:105B300006460025746A20684069C0F3C01594F8D1
:105B40004100212805D125B10020E084204600F045
:105B5000C8F820684069C0F3801594F842002228F4
:105B600005D125B10020E085204600F074F8606C76
:105B700040F0100060642046FDF74AFC70BD70B52F
:105B800005466C6A2868006800F02000002842D1B1
:105B9000E08500BF00BF21680C3151E8001F21F4EF
:105BA000807021680C3141E80002002AF3D100BF67
:105BB00000BF00BF2168143151E8001F21F001002F
:105BC0002168143141E80002002AF3D100BF00BF70
:105BD00000BF2168143151E8001F21F04000216806
:105BE000143141E80002002AF3D100BF202084F8DC
:105BF0004200206B01280ED100BF00BF21680C318C
:105C000051E8001F21F0100021680C3141E800022A
:105C1000002AF3D100BF00206063206B012804D16B
:105C2000A18D2046FDF74DFB02E02046FDF796FED4
:105C300070BD70B505466C6A01206063206B012859
:105C400005D1A08D41082046FDF73BFB02E0204630
:105C5000FDF78CFE70BD00BF00BF02680C3252E839
:105C6000002F22F4907102680C3242E80013002BDE
:105C7000F3D100BF00BF00BF0268143252E8002F0A
:105C800022F001010268143242E80013002BF3D124
:105C900000BF016B01290ED100BF00BF02680C32AA
:105CA00052E8002F22F0100102680C3242E8001383
:105CB000002BF3D100BF202180F8421000210163A6
:105CC000704710B504462068C06820F04000216885
:105CD000C860202084F841002046FDF7BDFE00206A
:105CE00010BD00BF00BF02680C3252E8002F22F046
:105CF000C00102680C3242E80013002BF3D100BF50
:105D0000202180F841107047F8B5044694F842000D
:105D1000222875D1A068B0F5805F0CD1206950B9F8
:105D20000025A66A20684068C0F308003080A06A99
:105D3000801CA06215E0A56A0026A068B0F5805F0F
:105D400003D0A06828B9206918B920684068287075
:105D500004E02068406800F07F002870A06A401CC2
:105D6000A062E08D401E80B2E085002846D1206808
:105D7000C06820F020002168C8602068C06820F456
:105D800080702168C8602068406920F001002168A7
:105D90004861202084F8420000206063206B0128C5
:105DA00026D10020206300BF00BF21680C3151E8DC
:105DB000001F21F0100021680C3141E80002002A88
:105DC000F3D100BF2068006800F0100010280AD14D
:105DD00000BF0020009020680068009020684068A4
:105DE000009000BF00BFA18D2046FDF76AFA02E0D7
:105DF0002046FDF7B3FD0020F8BD01E00020FBE7E1
:105E00000220F9E770B504462168096921F4405180
:105E1000E2681143226811612269A1681143626935
:105E200041EA02052168C96841F20C6291432943A5
:105E30002268D1602168496921F44071A269114347
:105E4000226851612D4A2168914202D1FCF772FD0E
:105E500001E0FCF75FFD00EBC00101EB001162689F
:105E60009200B1FBF2F100EBC00202EB001263689A
:105E70009B00B2FBF3F26423B2FBF3F202EBC2032A
:105E800003EB0212A1EB8201322202EB0111642228
:105E9000B1FBF2F101F0F00100EBC00202EB0012E5
:105EA00063689B00B2FBF3F26423B2FBF3F201EBF5
:105EB000021200EBC00101EB001163689B00B1FB13
:105EC000F3F100EBC00303EB00136668B600B3FB0D
:105ED000F6F36426B3FBF6F303EBC30606EB0313FA
:105EE000A1EB8301322303EB01116423B1FBF3F136
:105EF00001F00F0111442268916070BD003801402B
:105F000077B581B0044615460298A062A5850020A9
:105F10006064222084F842002848E16B88622848A7
:105F2000E16BC8622748E16B08630020E16B4863BE
:105F300002AE32682368191D2B46E06BFBF7B8FEF2
:105F400000BF002000902068006800902068406832
:105F5000009000BF00BF206970B100BF00BF216882
:105F60000C3151E8001F41F4807021680C3141E888
:105F70000002002AF3D100BF00BF00BF2168143126
:105F800051E8001F41F001002168143141E800028E
:105F9000002AF3D100BF00BF00BF2168143151E8CF
:105FA000001F41F040002168143141E80002002A3E
:105FB000F3D100BF002004B070BD00007F5B00087B
:105FC000335C00082F5B0008014691F8410021284E
:105FD00028D18868B0F5805F0BD1086948B90A6A92
:105FE0001088C0F308000B685860086A801C0862BB
:105FF00005E00B6A581C086218780B685860C88C5A
:10600000401E80B2C88458B90868C06820F080007B
:106010000B68D8600868C06840F040000B68D86022
:10602000002070470220FCE72DE9F04104460D46B0
:1060300017469846069E34E0701C88B32EB1FCF7D4
:1060400023F9A0EB0800B0422BD900BF00BF2168A4
:106050000C3151E8001F21F4D07021680C3141E867
:106060000002002AF3D100BF00BF00BF2168143135
:1060700051E8001F21F001002168143141E80002BD
:10608000002AF3D100BF202084F8410084F84200A8
:1060900000BF002084F8400000BF0320BDE8F0816D
:1060A000FFE7206800682840A84201D1012000E0F5
:1060B0000020B842C0D00020F0E7000008B51C481E
:1060C00000680068C0F3001068B300BF00200090B3
:1060D0001748006800680090154800684068009004
:1060E00000BF00BF1248FDF74EF912480068406833
:1060F000C0F5806010490880084602880F491048A2
:10610000FAF790F80C4802880C490E48FAF78AF81A
:106110004FF4806209490648FDF70AFC01200A494C
:1061200008700A4908700248FDF774F908BD0000BC
:1061300028480020B8480020860500207C37002031
:106140007C3300207C3B0020840500208505002056
:1061500010B50248FDF75EF910BD00007048002040
:1061600000BFFEE72DE9F04705460F4690460024A4
:10617000284600F025FBFBF7B7FE414885420CD1CD
:1061800017F808402246002301460120FBF754FE81
:1061900006460EB93B4804806EE03B4885420CD170
:1061A00017F808402246002301460120FBF744FE71
:1061B00006460EB935490C705EE0354885420CD173
:1061C00017F808402246002301460120FBF734FE61
:1061D00006460EB92F4804804EE02F48854202D073
:1061E0002E48854248D14FF43A762B4885421FD13C
:1061F0002B480088B04204DB29480088801B84B209
:1062000005E027480088301A84B244F4004422464E
:10621000002321490120FBF70FFE8146B9F1000F51
:1062200005D1C4F30E001F4908801F48048022E0F6
:106230001A4885421FD11D480088B04204DB1B4824
:106240000088801B84B205E018480088301A84B2A8
:1062500044F400442246002310490120FBF7ECFDE2
:106260008146B9F1000F05D1C4F30E001049088032
:106270001048048000BF00BFFBF7D4FDBDE8F087E5
:1062800000000708B600002000080708C100002031
:1062900000100708B80000200018070800200708B1
:1062A000E2000020E6000020D4000020E4000020EE
:1062B000E8000020D60000200FB4084B10B504A958
:1062C00002AA039800F03CF8044602A9002000F05E
:1062D000D8F9204610BC5DF814FB00008366000866
:1062E00002480068C0F30220704700000CED00E097
:1062F00010B5002804DB0A07130E054A135406E004
:106300000A07140E034A00F00F031B1FD45410BDDC
:1063100000E400E018ED00E002E008C8121F08C128
:10632000002AFAD170477047002001E001C1121F16
:10633000002AFBD1704700F0010181F313887047F8
:106340002DE9FF4F8BB088460546002606E025283C
:106350000BD0DDE90D1290476D1C761C28780028C3
:10636000F5D10FB03046BDE8F08F0024A146A2461B
:106370000122AE4900E0044315F8013F203B02FA38
:1063800003F00842F7D128782A2810D06FF02F02A6
:106390002878A0F13001092915D809EB890102EB11
:1063A000410144F0020400EB01096D1CF0E758F8CC
:1063B000041B5FEA010903D544F40054C9F1000944
:1063C00044F002046D1C28782E2817D115F8010F0F
:1063D00044F004042A280ED06FF02F022878A0F190
:1063E000300109290AD80AEB8A0102EB410100EBCE
:1063F000010A6D1CF2E758F804AB6D1C28786C2874
:106400000FD006DC4C2817D068280DD06A2814D18C
:1064100004E0742810D07A280FD10DE044F4001461
:106420000AE044F4801401E044F4401469788142A5
:1064300002D104F580146D1C6D1C2878692865D084
:1064400006DC00288DD0632827D0642806D15DE0C3
:106450006E2808D073282AD0752877D0DDE90D1270
:106460009047761CE0E0C4F30250022809D00328CC
:106470000DD0D8F8001004280DD00E6008F10408E3
:10648000D2E0D8F80010F217C1E90062F6E7D8F8B8
:1064900000100E80F2E70E70F0E718F8041B8DF87C
:1064A000001000208DF80100EB46012003E058F8B1
:1064B00004BB4FF0FF3061074FF0000701D40AE042
:1064C0007F1C57450DDA8742FADB1BF807100029BD
:1064D000F6D106E07F1C8742FCDB1BF80710002981
:1064E000F8D1DDE90D23A9EB07008146214600F034
:1064F000B1F83044C61904E0DDE90D121BF8010BB8
:1065000090477F1EF8D22146484688E058F8040B91
:10651000C4F302514FF00A0B032900D100B2042941
:1065200000D140B2002802DA40422D2102E02105CC
:1065300005D52B218DF82410012104E006E0E107A8
:1065400010D02021F6E708AF089113E058F8040BAB
:10655000C4F302514FF00A0B032900D180B2042981
:1065600000D1C0B20021EEE75946FAF73FF83031CA
:1065700007F8011D0028F7D1ADEB070000F1200B53
:10658000600702D524F4803401E04FF0010ADA45B7
:1065900002DDAAEB0B0000E00020824600EB0B01BD
:1065A00008980144A9EB01000A90E00306D4DDE954
:1065B0000D2321460A9800F04DF806444FF00009DB
:1065C00008E009A911F80900DDE90D12904709F169
:1065D0000109761C08998945F3DBE0030CD5DDE958
:1065E0000D2321460A9800F035F8064404E0DDE961
:1065F0000D1230209047761CBAF10001AAF1010A71
:10660000F5DC05E0DDE90D1217F8010B9047761C6B
:10661000BBF10001ABF1010BF4DC0A982146DDE986
:106620000D2300F005F806446D1C97E609280100CB
:106630002DE9F041044600251E461746880404D47F
:1066400005E039462020B0476D1C641EF9D5284668
:10665000BDE8F0812DE9F041044600251E46904634
:10666000C80301D5302700E02027880404D505E0C1
:1066700041463846B0476D1C641EF9D52846BDE832
:10668000F0810A68531C0B601070704730B50246E9
:106690000B464FF6FF70002110E0545C6040002470
:1066A00009E000F0010525B14AF2010585EA600024
:1066B00000E04010641C082CF3DB491C9942ECDB21
:1066C00030BD000010B504460B480068C06820F4D7
:1066D000005009490968C86007484460FDF70CF894
:1066E00008B1FAF744FA04480068C06840F4005062
:1066F00001490968C86010BD2848002010B54FF452
:1067000080610748F9F7A7FD4FF480610548F9F764
:10671000A2FD0020044908700449087010BD000063
:106720007C3B00207C37002085050020840500206C
:1067300010B50288C2F30323027863F31F12130615
:106740004288C2F3032464F31F1243EA024382889F
:10675000C2F3032464F31F1243EA0223C288C2F384
:10676000032464F31F1213430B6010BD30B50246BF
:106770000B460020002117E0545C80EA042000242E
:106780000EE000F400452DB141F2210585EA4005F7
:10679000A8B203E04FF6FF7505EA4000651CECB2B5
:1067A000082CEEDB4C1CA1B29942E5DB30BDC200E7
:1067B000002100BF01E000BF491C9142FBD370479C
:1067C00030B585B004460020019003940120049068
:1067D00000200090FBF788FB694601A8FBF7CAFA86
:1067E0000546FBF71FFB15BB1248844203D100206E
:1067F000114908801BE01148844203D10020104950
:10680000087014E00F48844204D14FF6FF700E491F
:1068100008800CE00D48844203D100200C49088018
:1068200005E00C48844202D100200B49088005B0E5
:1068300030BD000000000708B6000020000807086F
:10684000C100002000100708B80000200018070849
:10685000E600002000200708E80000202DE9FF4F97
:106860008BB08B4690469946199E0020089009F1FE
:10687000010258F8221058F82900F9F750FD824615
:106880006649F9F784FD07900A960A9EB00000F069
:1068900007FA04464FF0000A12E05046F9F727FEC7
:1068A00003900799F9F741FD049009F1010058F8A8
:1068B00020100498F9F7E1FC44F82A000AF1010AD3
:1068C000B245EADB4FF0FF35554806904FF0000A1D
:1068D00022E054F82A100B98F9F721FD0190F9F7FE
:1068E00041FE21F00041CDE90201F9F74EFE04908E
:1068F00006990498F9F766FE01D2504600E0284652
:10690000054606990498F9F75DFE01D2049800E067
:10691000069806900AF1010AB245DADB4148059073
:106920000996099EB00000F0BBF907464FF0000A37
:1069300011E05046F9F7DBFD3A490390F9F7F5FC11
:10694000049018985BF820100498F9F796FC47F823
:106950002A000AF1010AB245EBDB54F8250032495E
:10696000F9F73AFE04D248F29010304908804AE024
:1069700054F825002E49F9F72FFE1FD254F82500B0
:106980002949F9F71FFE19D857F82500F9F7EAFD4C
:1069900021F000410022274BCDE90001F9F735FD38
:1069A000CDE90201F9F7C5FD80B20890089840F4DE
:1069B000004008901D490898088024E054F82500FC
:1069C0001D49F9F709FE10D854F825001849F9F7C0
:1069D000F9FD0AD857F825001049F9F7A6FC8246B8
:1069E000F9F793FD114908800DE054F8250012498C
:1069F000F9F7E8FD04D240F21A400C49088002E0A1
:106A000000200A49088000200890384600F016F857
:106A1000204600F013F80FB0BDE8F08F00002041D1
:106A200000007A44CDCCCC3DB57DAA438005002042
:106A3000E9F70242000024408104153F10B5002808
:106A400021D0114B0022001F196803E0814203D8B6
:106A50000A4649680029F9D152B11368841A9C4248
:106A600004D1006818441060104602E0506000E055
:106A7000186039B102680B1A934203D10B681A44AB
:106A800002604968416010BD300600202DE9FC47D6
:106A900081460C461546AFB2264632483249086058
:106AA00007F50060C11700EB5151C9122F4A118040
:106AB0004FF400612E48F9F7CEFB2EA103C9CDE9B2
:106AC000000101202D49086044E0012211462C48B4
:106AD000FBF7D4FB0520FBF739F9002201212848F8
:106AE000FBF7CCFB4FF4006231462148FAF7F4F88B
:106AF0004FF480621C4801681D48FAF703F95020E2
:106B0000FFF755FE1D486A461EA103681F48FFF7A0
:106B1000D3FB80461FFA88F21C491D48FCF780FF12
:106B200006F500661048006800F500600E49086030
:106B3000012211461248FBF7A1FB0520FBF706F9DD
:106B4000002201210E48FBF799FB0C480068401C0D
:106B50000A49086009480068044909888842B4DD88
:106B6000BDE8FC87000002086800002064000020E7
:106B70000020002061636B3D000000006C000020DD
:106B8000000C014025732564000000007C330020C8
:106B90002848002070B5044672B6206880F3088843
:106BA00000BF6568A84770BDFBF780FBFEF7D6FE07
:106BB000FDF78EFCFDF724FCFDF74AFDFDF7DAFB3F
:106BC000FDF70EFDFDF760FD2448FCF7D1F92448E0
:106BD00000F02EFEFEF7C8FDF9F77CFE00F0BCFECB
:106BE000204800F05BFE204800F0E6FB1F4800F064
:106BF000DFFB054600F0D0FD1D4800F0D9FB05463F
:106C000000F000FE1BA11D48FFF756FB0446A2B290
:106C10001A491B48FCF704FF4FF4806219491848D1
:106C2000FCF786FE16480068C06840F01000144962
:106C30000968C860144801681448F9F789FE30B142
:106C4000002080F3138800BF1048FFF7A3FFFDF773
:106C500001FC00F067F800BFFEE7000034330020BD
:106C60000048070888F00708000007080008070820
:106C70000010070861707031000000007C330020B4
:106C8000284800207C37002058000020000002081F
:106C900001460020842901D0CA1C1044704700001E
:106CA000F0B50B30154D20F007010024144A0FE019
:106CB00003688B420BD38B4205D95E1A4318476891
:106CC000C3E9006700E04368136002C004E0021DEE
:106CD00010680028ECD12046002802D1286808B1AD
:106CE0000020F0BD064A07481060074A121A22F039
:106CF0000702C0E9002401202860D7E734060020FD
:106D000030060020E4560020E058002070B504460C
:106D100025460DB1294600E00121084600F038FF64
:106D2000002070BD10B500F061FF002010BD7FB5E0
:106D300004460D46606998B1A06988B1B4F90800AD
:106D4000FFF7A6FF0646D4E90510CDE900610290E1
:106D50002B462269D4E9001001F09CF8039013E05F
:106D6000B4F90800FFF794FF064603A8CDE90060D8
:106D7000238A9AB22B46D4E9001001F059F8012871
:106D800002D0002004B070BD0398FBE72DE9F0416C
:106D900005460E461C4807681C480068001D00F0A8
:106DA000FBFD50B91948006890F82C10012088406C
:106DB00017490968814316480160681C38B936B123
:106DC00012480168091D134800F030FE1AE07C19D2
:106DD0000E4800684460BC4207D20C480168091D97
:106DE0000D48006800F008FE0CE008480168091D25
:106DF0000A48006800F000FE09480068844201D299
:106E000007480460BDE8F081E4050020D0050020BB
:106E1000E8050020CC4A0020D8050020D405002039
:106E20000006002010B5044600F00CFE2348006860
:106E3000401C224908602248006840B9204804608C
:106E40000846006801280DD100F03AF90AE01D4813
:106E5000006838B91A480068C06AE16A884201D8F7
:106E60001748046018480068401C1749086094F8E7
:106E70002C1001208840154909680843134908600F
:106E8000E16A01EB8101124A02EB8100211D00F051
:106E9000CDFD00F001FE0B48006868B108480068AD
:106EA000C06AE16A884207D24FF080500949086001
:106EB000BFF34F8FBFF36F8F10BD0000E0050020C0
:106EC000D0050020EC050020FC050020E80500208E
:106ED000F049002004ED00E010B516E000F0B2FD2E
:106EE0000C48C068C468201D00F056FD0A480068C0
:106EF000401E0949086009480068401E07490860AB
:106F000000F0CAFD204600F00BF804480068002895
:106F1000E4D110BDB84A0020E0050020DC050020C7
:106F200010B5044694F8510030B9206B00F0D2FD42
:106F3000204600F0CFFD1AE094F85100012803D15B
:106F4000204600F0C7FD12E094F85100022801D15C
:106F5000012000E0002050B900BF502080F31188CC
:106F6000BFF34F8FBFF36F8F00BF00BFFEE710BDB1
:106F700030B54FF44063174800F007042CB1C01D32
:106F800020F00700134C041B1B1B0246124C22600E
:106F90000024114D6C60D018083820F007000F4C09
:106FA000206000240D4D2D686C600C4D2D682C6008
:106FB0001146441A4C60094C24680C60084D4C681A
:106FC0002C60084D4C682C604FF00044064D2C603E
:106FD00030BD0000E04A00200C060020140600200E
:106FE0001C060020180600202006002000BFFFF726
:106FF00073FF064800680128F9D94FF08050044912
:107000000860BFF34F8FBFF36F8FF0E7F0490020A8
:1070100004ED00E02DE9FF5F81460F469246DDE971
:107020000E6B109CAAF10100216B01EB800828F087
:10703000070808F0070008B9012000E0002050B957
:1070400000BF502080F31188BFF34F8FBFF36F8FC5
:1070500000BF00BFFEE7002507E0795D04F13400C2
:107060004155785D00B902E06D1C102DF5D300BFCD
:10707000002143200155072E00D30626E6626664F0
:107080000020A064201D00F0B4FC04F1180000F002
:10709000B0FC2461C6F10700A06164620020E064D6
:1070A00084F8500049464046039A00F049F92060B0
:1070B000BBF1000F01D0CBF80040BDE8FF9F0000FE
:1070C00010B5002407E004EB84010F4A02EB8100B5
:1070D00000F082FC641C072CF5D30C4800F07CFC0B
:1070E0000B4800F079FC0B4800F076FC0A4800F0F1
:1070F00073FC0A4800F070FC044809490860044821
:107100000849086010BD0000F04900207C4A0020BA
:10711000904A0020A44A0020B84A0020CC4A00200F
:10712000D4050020D805002010B50146164800E01F
:10713000006803688B42FBD30246436813448B42CA
:1071400004D143684C682344436001460A464B68B7
:1071500013440468A34211D10C4C03682468A34271
:1071600008D04B680468646823444B6003681B685C
:107170000B6005E0054B1B680B6001E003680B60CA
:10718000884200D0016010BD0C06002014060020CB
:107190000A490968096809B9012100E0002121B103
:1071A0004FF0FF31064A116006E004490968C968DA
:1071B000C868034A4168116070470000D405002088
:1071C000000600200E480068401C08B9012000E0BD
:1071D000002050B900BF502080F31188BFF34F8FBB
:1071E000BFF36F8F00BF00BFFEE700BF502080F3EA
:1071F0001188BFF34F8FBFF36F8F00BF00BFFEE753
:10720000240600202DE9F04104464FF0000800F06C
:1072100045FD4648006808B9FFF7AAFE44480068E3
:10722000204000286BD1D4B1083404F00700B0B17D
:1072300004F00700C0F10800044404F0070008B996
:10724000012000E0002050B900BF502080F31188D9
:10725000BFF34F8FBFF36F8F00BF00BFFEE7002C5F
:107260004DD034480068844249D8334E30460568D2
:1072700001E02E462D686868A04202D228680028E6
:10728000F7D12A480068854239D0306800F10808F3
:10729000286830606868001B102819D92F1907F07A
:1072A000070008B9012000E0002050B900BF5020BD
:1072B00080F31188BFF34F8FBFF36F8F00BF00BF04
:1072C000FEE76868001B78606C603846FFF72CFFAB
:1072D000184968680968081A16490860084600686D
:1072E00016490968884203D21248006813490860A9
:1072F0000F4968680968084368600020286000F04A
:10730000C9FE08F0070008B9012000E0002050B9CC
:1073100000BF502080F31188BFF34F8FBFF36F8FF2
:1073200000BF00BFFEE74046BDE8F0811406002024
:1073300020060020180600200C0600201C06002055
:10734000001F4FF080730360001F21F001030360F2
:10735000001F034B036014380260203870470000A0
:10736000C571000810B50548FBF7ACFF4FF480620B
:1073700003490248FCF7DCFA10BD00002848002051
:107380007C37002002460948006838B1002002E03E
:107390000B5C1354401C0528FADB06E0002002E0D9
:1073A0000B5C1354401C0428FADB704734000020A7
:1073B000014608887047000010B504462046FFF7D4
:1073C000F7FF03464FF6FF70834204D1034800885D
:1073D0000249088001E00148038010BDB60000208A
:1073E0002DE9FE4F06460F4690461D46DDE90C9AF4
:1073F0000E9C0020009001900290F0B28DF80000E9
:107400008DF801708DF8028028128DF80300E8B223
:107410008DF804004FEA29208DF8050009F0FF00DF
:107420008DF806004FEA2A208DF807000AF0FF00C9
:107430008DF80800A01EC1B26846FFF727F9834601
:107440000BF0FF01A01E0DF800104FEA2B21601E6B
:107450000DF80010631EA2B269460448FCF787FAD3
:10746000FFF74CF9FFF77EFFBDE8FE8F28480020AC
:107470002DE9F04F85B006460F4690461D46DDE9E2
:107480000FABDDF83890119C002001900290039022
:107490000490F0B28DF804008DF805708DF8068028
:1074A00028128DF80700E8B28DF808004FEA29206D
:1074B0008DF8090009F0FF008DF80A004FEA2A2034
:1074C0008DF80B000AF0FF008DF80C004FEA2B201E
:1074D0008DF80D000BF0FF008DF80E00A01EC1B25C
:1074E00001A8FFF7D3F800900098C1B2A01E01AA2E
:1074F000115400980112601E1154631EA2B201A91A
:107500000448FCF734FAFFF7F9F8FFF72BFF05B052
:10751000BDE8F08F284800202DE9F04F85B00646E1
:107520000F4690461D46DDE911B4DDE90E9A0020B4
:107530000190029003900490F0B28DF804008DF851
:1075400005708DF8068028128DF80700E8B28DF8D6
:1075500008004FEA29208DF8090009F0FF008DF896
:107560000A004FEA2A208DF80B000AF0FF008DF880
:107570000C00109800128DF80D001098C0B28DF814
:107580000E004FEA2B208DF80F000BF0FF008DF856
:107590001000A01EC1B201A8FFF778F80090009873
:1075A000C1B2A01E01AA115400980112601E11540C
:1075B000631EA2B201A90548FCF7D9F9FFF79EF8AE
:1075C000FFF7D0FE05B0BDE8F08F0000284800208E
:1075D0002DE9FC4706460F4690461D460A9C0020B2
:1075E00000900190F0B28DF800008DF801708DF8D8
:1075F000028028128DF80300E8B28DF80400A01E66
:10760000C1B26846FFF742F8814609F0FF01A01EAB
:107610000DF800104FEA2921601E0DF80010A2B2EB
:10762000234669460448FCF7A2F9FFF767F8FFF71D
:1076300099FEBDE8FC870000284800202DE9FC41A8
:107640000746884614461D46002000900190F8B277
:107650008DF800008DF8018020128DF80200E0B254
:107660008DF8030028128DF80400E8B28DF80500AB
:1076700006216846FFF70AF80646F0B28DF80600C4
:1076800030128DF807000723082269460448FCF7EA
:107690006EF9FFF733F8FFF765FEBDE8FC810000E7
:1076A000284800202DE9FE4F06460F4690461D460D
:1076B000DDE90C940020009001900290F0B28DF86A
:1076C00000008DF801708DF8028028128DF80300FB
:1076D000E8B28DF804004FEA29208DF8050009F082
:1076E000FF008DF80600A01EC1B26846FEF7CEFF6F
:1076F00082460AF0FF01A01E0DF800104FEA2A2171
:10770000601E0DF80010631EA2B269460448FCF723
:107710002EF9FEF7F3FFFFF725FEBDE8FE8F000010
:10772000284800202DE9FE4306460F4614461D4614
:10773000DDF828900020009001900290F0B28DF8C2
:1077400000008DF8017020128DF80200E0B28DF873
:10775000030028128DF80400E8B28DF805008DF8BA
:10776000069007216846FEF791FF804608F0FF006B
:107770008DF807004FEA28208DF8080009231A46E3
:1077800069460448FCF7F3F8FEF7B8FFFFF7EAFD97
:10779000BDE8FE832848002010B504464FF6FF7070
:1077A000844214D1002208211548FAF767FD00220F
:1077B00010211348FAF762FD002220211048FAF741
:1077C0005DFD002240210E48FAF758FD17E004F055
:1077D000010208210A48FAF751FDC4F340021021C2
:1077E0000748FAF74BFDC4F3800220210448FAF75A
:1077F00045FDC4F3C00240210148FAF73FFD10BD2A
:10780000000C014010B50446072C04DC074951F870
:107810002400FEF757FF4FF6FF70844201D0032C7F
:1078200003D14FF41650FEF74DFF10BDA005002008
:1078300010B50446022221461648F9F74DFA0020F9
:107840000FE0144931F810104FF47F4202EA012191
:10785000104A32F8102041EA12210E4A22F8101084
:10786000401C0128EDDB0B4800884FF6FF71884271
:1078700003D10020084908600BE0064800884FF457
:107880007F4101EA00200349098840EA11200249AA
:10789000086010BD980500202800002038B5044677
:1078A000082212491248F9F717FA00200FE0104990
:1078B00031F810104FF47F4202EA01210C4A32F8ED
:1078C000102041EA12210A4A22F81010401C042814
:1078D000EDDB69460648FEF72BFF0098401C00B917
:1078E00038BD04490098086000BFF9E788F0070830
:1078F00006000020BC00002010B5044604222146EA
:107900000B48F9F7E9F90A4840880949098840EA2B
:1079100001400849086008460068401C10B9002072
:10792000086004E00348006880300249086010BD28
:10793000420000203C00002010B504460222211D18
:107940000348F9F7C9F9024800880249088010BDC8
:10795000460000204000002010B510220C490D48C0
:10796000F9F7BAF900200FE00A4931F810104FF486
:107970007F4202EA0121074A32F8102041EA12212F
:10798000044A22F81010401C0828EDDB10BD00004E
:10799000005007089A06002001460A69D1E9013023
:1079A0009860D1E9010358605068884201D1886825
:1079B0005060002008611068401E10601068704719
:1079C000034B0360034B0B60802313607047000080
:1079D000E03000203431002000F1080141604FF018
:1079E000FF31816000F10801C16001610021016087
:1079F000704700210161704710B502460B685C1C9E
:107A00000CB9106907E002F1080000E04068446822
:107A100024689C42FAD944684C604C68A160886034
:107A200041600A611468641C146010BD42684A60B9
:107A300093688B60936859609160086103685B1C70
:107A40000360704700BF502080F31188BFF34F8F51
:107A5000BFF36F8F00BF0E480068401C0C490860E0
:107A600008460068012812D10A480068C0B208B967
:107A7000012000E0002050B900BF502080F31188A1
:107A8000BFF34F8FBFF36F8F00BF00BFFEE770479C
:107A90002406002004ED00E00D48006850B900BF46
:107AA000502080F31188BFF34F8FBFF36F8F00BF5B
:107AB00000BFFEE706480068401E0549086008460A
:107AC000006820B9002080F3118800BF00BF704714
:107AD0002406002070B506463546002E3FD0083DEE
:107AE0002C461F4960680968084008B1012000E081
:107AF000002050B900BF502080F31188BFF34F8F92
:107B0000BFF36F8F00BF00BFFEE7206808B90120F8
:107B100000E0002050B900BF502080F31188BFF36F
:107B20004F8FBFF36F8F00BF00BFFEE70C49606847
:107B30000968084098B1206888B9094960680968EF
:107B40008843606000F0AAF8064960680968084444
:107B5000044908602046FFF7E7FA00F09BFA70BD81
:107B6000200600201806002000204FF0E0210861C8
:107B70008861064800684FF47A71B0FBF1F0401E4E
:107B80004FF0E0214861072008617047CC050020D4
:107B900070B504460025D4B11248006808B9012028
:107BA00000E0002050B900BF502080F31188BFF3DF
:107BB0004F8FBFF36F8F00BF00BFFEE700F06EF87E
:107BC00000212046FFF7E2F800F064FA05463DB9CF
:107BD0004FF0805004490860BFF34F8FBFF36F8FA1
:107BE00070BD00000806002004ED00E010B586B06E
:107BF00000200590049003AA04A905A8FFF7E0FE61
:107C00000022DDE904101346CDE9002102901CA1F9
:107C10001D48039A00F03EF91C49086008460068B8
:107C200008B1012400E00024012C15D100BF502030
:107C300080F31188BFF34F8FBFF36F8F00BF4FF0FA
:107C4000FF301349086001201249086000201249E2
:107C5000086000F071F810E0601C08B1012000E03D
:107C6000002050B900BF502080F31188BFF34F8F20
:107C7000BFF36F8F00BF00BFFEE706B010BD00006E
:107C800049444C4500000000ED6F00080406002048
:107C900000060020EC050020E405002002480068F2
:107CA000401C014908607047080600201D48006814
:107CB00018B101201C49086032E000201A49086010
:107CC0001A480068B0FA80F0C0F11F0101EB810092
:107CD000174A52F8200008B1012000E0002050B9F6
:107CE00000BF502080F31188BFF34F8FBFF36F8F19
:107CF00000BF00BFFEE701EB81020D4B03EB8200EA
:107D000042685268426000F108024368934202D11F
:107D10004268526842604268D268064B1A6000BFEF
:107D20007047000008060020F4050020E805002048
:107D3000F0490020D00500201CB5384908460078DD
:107D40000190FF200A4610700846007800909DF8C8
:107D5000000000F0F0009DF80020904201D10120C9
:107D600000E0002050B900BF502080F31188BFF31D
:107D70004F8FBFF36F8F00BF00BFFEE79DF800007D
:107D800000F05000264A10700720264A106009E0D3
:107D900024480068401E234A10609DF800004006F9
:107DA000000E00909DF8000000F080008028EFD0C9
:107DB0001C480068C0F10700042801D1012000E040
:107DC000002050B900BF502080F31188BFF34F8FBF
:107DD000BFF36F8F00BF00BFFEE7124800680002CC
:107DE000104A10601046008800F4E06010600B4AF2
:107DF000019810700C48006840F470000A4908604F
:107E00000846006840F070400860FFF7ADFE0020B3
:107E100006490860F8F7AAF900201CBD00E400E05C
:107E2000280600202C06002020ED00E0240600207B
:107E30002DE9FF4F85B0804689461746DDE912AB34
:107E4000B800FFF7DFF9064656B15420FFF7DAF91C
:107E500004460CB1266304E03046FFF73BFE00E029
:107E600000248CB1002084F85100CDE900ABCDE9AD
:107E700002403A4649464046089BFFF7CBF8204669
:107E8000FEF7D0FF012501E04FF0FF35284609B08D
:107E9000BDE8F08F2DE9F04F85B007468846914642
:107EA0009A46DDE90EB6109C0EB1012000E00020DC
:107EB00050B900BF502080F31188BFF34F8FBFF33C
:107EC0006F8F00BF00BFFEE70CB1012000E0002073
:107ED00050B900BF502080F31188BFF34F8FBFF31C
:107EE0006F8F00BF00BFFEE7542003900398542813
:107EF00001D1012000E0002050B900BF502080F3E4
:107F00001188BFF34F8FBFF36F8F00BF00BFFEE735
:107F1000B4B1AEB125462C462E63022085F851003F
:107F2000002004A953464A46CDE900B1CDE90250EC
:107F300041463846FFF76EF82846FEF773FF01E02A
:107F400000200490049805B0BDE8F08F2DE9F041C1
:107F50004FF0000844480068002877D14348006883
:107F6000451C4248056015BB41480068006808B9D7
:107F7000012000E0002050B900BF502080F311889C
:107F8000BFF34F8FBFF36F8F00BF00BFFEE73848CE
:107F90000768384800683649086036480760364840
:107FA0000068401C34490860FFF7F2F800BF33480E
:107FB000006885423CD300BF2D480068006808B9BE
:107FC000012000E0002020B14FF0FF302B49086075
:107FD0002DE027480068C068C4686668B54202D2D0
:107FE0002648066023E0201DFFF7D6FCA06A18B1E2
:107FF00004F11800FFF7D0FC94F82C100120884001
:108000001F49096808431E490860E16A01EB8101C4
:108010001C4A02EB8100211DFFF708FD1A49E06AA6
:108020000968C96A8842C7D34FF00108C4E700BF96
:1080300015480068C06A00EB8000124951F8200022
:10804000012801D94FF0010805E0FFE70F4800685B
:10805000401C0E4908600E48006808B14FF0010846
:108060004046BDE8F081000008060020E40500203D
:10807000D4050020D8050020F805002000060020C7
:10808000E8050020F0490020D0050020F005002080
:10809000F405002070B5002400263648006850B969
:1080A00000BF502080F31188BFF34F8FBFF36F8F55
:1080B00000BF00BFFEE7FFF7C5FC2E480068401E6A
:1080C0002C4908600846006800284FD12A480068FB
:1080D00000284BD024E02948C068C46804F1180087
:1080E000FFF75AFC201DFFF757FC94F82C100120D5
:1080F000884023490968084321490860E16A01EB87
:108100008101204A02EB8100211DFFF78FFC1E49EF
:10811000E06A0968C96A884202D301201B490860E5
:108120001648006808B9012000E000200028D2D0DD
:108130000CB1FFF72DF81648056865B100BFFFF7D1
:1081400005FF10B10120114908606D1E002DF6D108
:1081500000200F4908600D48006838B1012630073B
:108160000C490860BFF34F8FBFF36F8FFFF794FC8C
:10817000304670BD08060020E0050020A44A00201B
:10818000E8050020F0490020D0050020F40500207B
:10819000F005002004ED00E06572726F72000000CF
:1081A000000801400100000000080140020000003A
:1081B0000008014004000000000801400800000021
:1081C00000080140100000000008014020000000ED
:1081D000000801404000000000080140800000004D
:1081E000B0820008C1580008030000000000000031
:1081F0008000000000000000000000008C820008E9
:108200000957000803000000000000008000000083
:108210000000000000000000988200085557000888
:1082200003000000000000008000000000000000CB
:1082300000000000A48200085F570008030000004F
:1082400000000000800000000000000000000000AE
:1082500002030405060708090A0B0C0D0E0F101087
:10826000010202030405060708090A0B0C0D0E0F94
:1082700010100102000000000000000001020304D1
:108280000607080900000000010203046D7954612B
:10829000736B3032000000006D795461736B3033C2
:1082A000000000006D795461736B303400000000F1
:1082B0006961705461736B00D8820008000000206F
:1082C00038060000820700080887000838060020EA
:1082D000A856000028630008017002458062C104AE
:1082E0002E1008232320C21A1C041A18041A14047E
:1082F0001A10041A0C041A08041A04041119041A96
:10830000F85D1AF0041AE8041AE0041AD8041AD026
:10831000041AC8041AC0041AB8041AB0041AA8042B
:108320001AA0041A98041A90041A88041A80041ACD
:1083300070041A60041A50041A40041A30041A20F7
:10834000042A10B529541AC04819041AA0041A8026
:10835000041A400411290C62BF33803F1A400319EC
:10836000041A80041AA0041AC0041AE004111A4165
:108370004819041A20041A30041A40041A50041A26
:1083800060041A70041A80041A88041A90041A9857
:10839000041AA0041AA8041AB0041AB8041AC004D3
:1083A0001AC8041AD0041AD8041AE0041AE8041AE5
:1083B000F0041AF8041122421A04041A08041A0CD0
:1083C000041A10041A14041A18041A1C041A20049B
:1083D0001A24041A28041A2C041A30041A34041A11
:1083E00038041A3C041A40041A44041A48041A4C6B
:1083F000041A50041A54041A58041A5C041A60042B
:108400001A64041A68041A6C041A70041A74041AA0
:1084100078041A7C041A80041A82041A84041A86C6
:10842000041A88041A8A041A8C041A8E041A9004F6
:108430001A92041A94041A96041A98041A9A041A9E
:108440009C041A9E041AA0041AA2041AA4041AA6D0
:10845000041AA8041AAA041AAC041AAE041AB00426
:108460001AB2041AB4041AB6041AB8041ABA041ACE
:10847000BC041ABE041AC0041AC2041AC4041AC6E0
:10848000041AC8041ACA041ACC041ACE041AD00456
:1084900000FF00D242CC76AA4348709F43EB32954E
:1084A0004324AF8B43A5D68243A13875433EE8658C
:1084B0004318A65743D95D4A43E0FC3D431372324B
:1084C00043A5AD274313A11D43FA3E14430F7B0B75
:1084D00043EF4903434142F742FAEDE8421F85DB8F
:1084E000423FF7CE421835C3427D30B8426ADCAD18
:1084F00042E72CA442A1169B42428F9242438D8AAE
:1085000042A107834271EC774282A26A4254235E01
:1085100042B16152424E514742B5E63C423F1733A9
:108520004217D92942EB2221423DEC18420E2D116F
:108530004201DE0942E9F7024210E9F841719BEC81
:1085400041B3FBE0412EFFD541439CCB4186C9C1DD
:1085500041917EB84133B3AF41D95FA741BF7D9F01
:1085600041F00598417CF29041713D8A41B1E1832F
:108570004168B37B41F24170416666654159175BC2
:1085800041D34D51410C0248410E2D3F414BC8365D
:108590004120099FCD2E414C3727411015204168BD
:1085A000221941029A12417C610C418E750641B735
:1085B000D118F9418FE4F6401EA7EC408FE4E24069
:1085C0005396D940AEB6D040143FC8406B2BC04044
:1085D000C976B840A01AB1407B14AA409E5EA34061
:1085E000C3F59C40D0D596407FFB9040B7628B404E
:1085F000D50986401CEB80401B0D78407DAE6E4057
:1086000017B76540A3235D40EEEB5440B30C4D40DB
:108610004D8445408C4A3E40705F37400EBE30402E
:108620007C612A4017482440986E1E405BD3184056
:108630007671134045470E40835109408A8E0440AD
:1086400072F9FF3F9031F73F27C2EE3FA9A4E63F02
:108650005DDCDE3F705FD73FE02DD03F2041C93F5A
:108660003199C23FCA32BC3FA60AB63F7E1DB03F19
:108670000A68AA3F4BEAA43FF9A09F3FCE889A3FE1
:10868000CBA1953FA7E8903F1D5A8C3F72F9873FD9
:108690001AC0833F9B557F3FA779773F57EC6F3FC9
:1086A000029A683FC58F613F83C05A480033105417
:1086B0003F0DE04D3FBEC1473FDCD7413FF6283C70
:1086C0003FF0A7363FCA54313F11362C3FAB3E270F
:1086D0003F2575223FF2D21D3F1058193F810415E6
:1086E0003F5AFF01C123B00423600923C012338025
:1086F00025324B329632E153C2013210390A03550A
:0887000024F41AAA0101100083
:0400000508000131BD
:00000001FF
